:10000000E8430020758C000001CA011001CA0110EC
:1000100001CA011001CA011001CA011001CA011070
:1000200001CA011001CA011001CA011001CA011060
:0C00300001CA011001CA01103FCA0110F2
:10003C00F3010100012002A80700201712000100A3
:10004C0002C80600205200015200011200010002F9
:04005C000800000098
:100100003C0000000000000000000000340100007E
:1001100000000000000000000100000000000000DE
:1001200000000000000000000000000001000000CE
:0C013000000000000800000000000000BB
:10013C003400000000000000000000006801000016
:10014C0000000000000000000100000000000000A2
:10015C00010000000000000000000000080000008A
:04016C00000000008F
:1001700030000000000000000000000098010000B6
:10018000040000000000000001000000FFFFFFFF6E
:10019000FF00000001000000080000000000000057
:1001A0002C0000000000000000000000C40100005E
:1001B000040000000000000001000000FFFFFFFF3E
:0C01C000FFFFFFFF08000000000000002F
:1001CC0034050000E401000099A1011095A701106D
:1001DC00A5C2011009B2011045B8011000000000C1
:0801EC00000000002E000000DD
:1001F40028000000000000000000000014020000BD
:100204000000000000000000FFFFFFFF00000000EE
:080214000800000000000000DA
:10021C00300500003002000069C201106DC10110F0
:10022C001FC2011095BA0110000000000000000070
:04023C00300000008E
:10024000300500005402000075C20110A9B601106B
:100250009DBF011049B60110000000000000000021
:040260003100000069
:1002640024000000000000000000000080020000E4
:100274000000000000000000000000000800000072
:040284000000000076
:10028800240000000000000000000000A40200009C
:10029800000000000000000000000000080000004E
:0402A8000000000052
:1002AC00240000000000000000000000C802000054
:1002BC000000000001000000000000000800000029
:0402CC00000000002E
:1002D000000000004C0900200400000000000000A5
:1002E000000000002000000070010000300000004D
:1002F0001C0200005409002004000000000000005F
:10030000000000000C000000300400001800000095
:10031000400200005C090020040000000000000012
:100320000000000024000000480400001800000045
:10033000000000006409002004000000000000002C
:100340000000000010000000A00100002C000000D0
:10035000CC0100006C090020040000000000000037
:1003600000000000200000006402000024000000E3
:10037000FFFFFFFF740900200400000000000000E0
:100380000000000028000000880200002400000097
:10039000FFFFFFFF840900200400000000000000B0
:1003A00000000000580000003C0100003400000084
:1003B000FFFFFFFF8C090020040000000000000088
:1003C00000000000100000006004000018000000A1
:1003D000FFFFFFFF94090020040000000000000060
:1003E000000000001C000000AC020000240000001F
:1003F000FFFFFFFF9C090020040000000000000038
:100400000000000038000000F40100002800000097
:10041000FFFFFFFFA409002004000000000000000F
:100420000000000054000000000100003C0000003B
:100430001800000000000000000000004004000060
:080440000800000000000000AC
:100448001800000000000000000000005804000030
:08045800080000000000000094
:100460001800000000000000000000007004000000
:0804700008000000000000007C
:0804780001000000288E0000C5
:040484000100000073
:0404880000000C0064
:04048C0000000D005F
:040490003200000036
:040494000200000062
:0404980048070020F1
:04049C00000200005A
:0404A0000000000058
:0404A40001CA011078
:0404A8000000000050
:0404AC00000000004C
:0404B0000800000040
:0404B4000000200024
:0404B8001007002009
:0404BC00010000003B
:0404C000E808002028
:0404C400080000002C
:0404C8000000000030
:0404CC00000000002C
:0404D0000000000028
:0404D4000000000024
:0404D8000000000020
:0404DC00010000001B
:0404E0007807002079
:0404E400060000000E
:0404E800010000000F
:0404EC007C0600206A
:0404F0000000000008
:0404F4000000000004
:0404F80000020000FE
:0404FC0000000000FC
:020502002A00CD
:020504000100F4
:020506002500CE
:020508003000C1
:02050A003100BE
:02050C002E00BF
:02050E000100EA
:0105100001E9
:0805140004000000F08C00005F
:08051C000000000000000000D7
:0405240000000100D2
:0405280000000300CC
:04052C0087C401106F
:04053000380500008A
:040534003805000086
:0405380000000000BF
:04053C00800000003B
:040540008000000037
:0405440000000000B3
:04054800E80800209F
:04054C00131E00007A
:040550002000000087
:040554008C8C00008B
:040558007CF701002B
:04055C000DC30110BA
:040560008D150000F5
:040564008F150000EF
:0405680099C801101D
:04056C009BC8011017
:040570000000000087
:04057400222300003E
:0405780024F6010064
:04057C003CF6010048
:040580000CF6010074
:0205840008006D
:0205860009006A
:02058800010070
:02058A0000006F
:01058C00016D
:040590000000000067
:040594000000000063
:04059800000000005F
:04059C00000000005B
:0405A000291400001A
:0405A40089140000B6
:0405A8000913000033
:0405AC00B314000084
:0405B00071130000C3
:0405B4002713000009
:0405B800B11300007B
:0405BC00F514000032
:0405C000911D000089
:0405C400931F000081
:0405C800971F000079
:0405CC000800000023
:0405D0002400000003
:0405D400180000000B
:0405D80028000000F7
:0405DC0020000000FB
:0405E0003C000000DB
:0405E4000C00000007
:0405E80034000000DB
:1005EC00DFF800F0F5C00110DFF800F049BA011097
:1005FC00DFF800F0E5C10110DFF800F025C20110B2
:10060C00DFF800F0C1C20110DFF800F0E3BF011009
:10061C00DFF800F013C10110DFF800F0B5C10110D4
:10062C00DFF800F0D5C20110DFF800F0F5B80110CA
:10063C00DFF800F0D5C00110DFF800F0F1C50110B3
:10064C00DFF800F095C00110DFF800F00DA80110E4
:10065C00DFF800F0BDBE0110DFF800F021C1011081
:10066C00DFF800F0A5B90110DFF800F021BA011095
:10067C00DFF800F0BDC20110DFF800F015B6011074
:10068C00DFF800F019A70110DFF800F02DBF011002
:10069C00DFF800F0E1B50110DFF800F0D9C201106D
:1006AC00DFF87C02007D704738B5DFF87C02DFF89C
:1006BC0074520068EFF3118480F31188A86800214C
:1006CC00FFF7BEFF6969081AA969814238BF00208B
:1006DC0084F3118832BD00002DE9F041DFF84802A7
:1006EC00DFF840420768EFF3118887F31188A068A0
:1006FC000121FFF7A5FF0121A1830021E183656999
:10070C0021682268461B801A691A884204D200208C
:10071C00A08388F311882AE088F31188002005E073
:10072C004519361A29460120FFF78EFF8642F7D26B
:10073C00EFF3118887F31188E18B012903D1294646
:10074C000020FFF781FFA16910F1010F08BF0846D7
:10075C0003D0801B814238BF08464119FFF778FF50
:10076C00012020840020A083256088F31188BDE837
:10077C00F081808A70470021DFF8B0210160126897
:10078C001044FFF751BF000038B500F0D3F8EFF379
:10079C00118580F31188207C022808D12046FFF7B0
:1007AC005BFF002020742946A068FFF759FF85F3F2
:1007BC00118831BD03681A4003680B408B4208BF97
:1007CC000A4312B101689143016010467047000062
:1007DC002DE9F0431F4617F1010F18BF002F91B000
:1007EC0004460D4616460AD06B463A46DFF84011D1
:1007FC0008A8FFF739FF08A80390022002E00020A8
:10080C00039003208DF8100006950796FFF7F0FE75
:10081C0002903246DFF81001D0F80080EFF3118916
:10082C0088F3118829462046FFF7C4FF050007D03E
:10083C00039808B1FFF71CFF89F31188284633E0B1
:10084C001FB989F3118800202EE0FFF7C9FE054679
:10085C000299DFF8D800C1F818D069460068204426
:10086C00FFF7DAFE0298FFF707FF9DF81000022849
:10087C0004BF0398FFF704FF89F311882846FFF79C
:10088C00B3FEEFF3118488F31188039818B1FFF7C6
:10089C00EFFE0020039000200299886184F31188F8
:1008AC009DF8100000B1059811B0BDE8F083000070
:1008BC00F8B50446DFF874000068261800F03BF821
:1008CC00EFF3118580F311882068084320603046CF
:1008DC00FFF79EFE10B185F31188F1BDFFF780FE86
:1008EC0007463046FFF79CFE0646F269B169204682
:1008FC00FFF760FF706160B13046FFF7ADFE01207D
:10090C003074F06808B1FFF777FEB0682946FFF73E
:10091C00A7FE85F311883846BDE8F240FFF764BEA8
:10092C00A4010020780100201C8E0000248E000001
:10093C009507000004460148006870471C8E0000B3
:10094C00DFF80410096870471C8E000000F01ABE16
:10095C0080B5002301223421DFF8F00901F0D0F832
:10096C0000B10120C0B202BDDFF8C41A0A68002829
:10097C0012BF42F0010050084000086070470000B0
:10098C007047FEE710B582B0042001F0F1F80228A0
:10099C0018BF03280DD1032000901C234FF04052A8
:1009AC000021DFF8A80901F088F8BDE81640042002
:1009BC006AE0DFF89C19DFF89C0A09684418DFF834
:1009CC009419DFF8940A0968B0FBF1F12046FFF79F
:1009DC0017FE2046BDE81640FFF716BE80B5DFF8BF
:1009EC0078090078DFF8740901688908890041F0FA
:1009FC000101016001F0C9F801F053F9DFF8601949
:100A0C00002008600220DFF894190968C96888473B
:100A1C00DFF85C0A016849084900016000F01BFA24
:100A2C00042000F013F900F0B6BC0000DFF82C1A1B
:100A3C00085C70470022012904D1012807D1DFF896
:100A4C00600903E0012802D1DFF82C0A0268104685
:100A5C007047DFF8000A00797047000001F0AAB86F
:100A6C0010B5DFF83C160968EFF3118481F3118897
:100A7C00DFF8E019C9880120012908BFFFF768FFDA
:100A8C0084F3118810BD000030B5DFF81416DFF8C0
:100A9C0088390A68EFF3118182F31188B0FA80F279
:100AAC00C2F11F029A5CB0FA80F4C4F11F04551E07
:100ABC001D5505D1DFF89C29136823EA000010604E
:100ACC0081F3118830BD00002DE9F041FFF738FFAC
:100ADC00EFF3118481F31188DFF880190A5C531E3F
:100AEC000B5444D1DFF87819DFF8788901EB8005D5
:100AFC002E786F88300618D5D8F80010096A384659
:100B0C008847D8F80010896A38468847D8F800100A
:100B1C00096B38468847DFF8501901200860DFF868
:100B2C004C0900688007FAD514E0700606D5DFF88A
:100B3C00AC1951F82710002088470BE0D8F80010AA
:100B4C00896938468847D8F80010496B3846884779
:100B5C000228F8D106F03F003F2818BFFFF7B4FF7A
:100B6C00687800F03F003F2818BFFFF7ADFF84F313
:100B7C001188BDE8F08110B508B1140001D1032033
:100B8C0010BD8160C26003610146DFF8E828DFF820
:100B9C00500912681044FFF777FD002010BD0000CB
:100BAC00F8B50446DFF8F804DFF8B0180068EFF386
:100BBC00118580F311880A5D531C0B55002A3ED118
:100BCC00DFF89C1801EB8407387800F03F003F28D1
:100BDC0018BFFFF7E5FF787800F03F003F2818BFFB
:100BEC00FFF7DEFF7E883878DFF87878010613D5BA
:100BFC003968C969304688473968496A3046884738
:100C0C003968C96A3046884700F038F8DFF85C0864
:100C1C0000688007FAD512E0400606D5DFF8BC184C
:100C2C0051F826100120884709E039684969304697
:100C3C0088473968496B304688470128F9D185F3D4
:100C4C0011882046BDE8F24001F08AB9DFF8501453
:100C5C000A68EFF3118182F31188DFF8F827136823
:100C6C0003431360B0FA80F0C0F11F00DFF8A8272F
:100C7C00135C5B1C135481F311887047DFF8E81781
:100C8C0001200860704700002DE9F04F4FF000087C
:100C9C000021012883B0C1468A4618BF022412D114
:100CAC00DFF8FC03DFF838780268EFF3118082F389
:100CBC0011883A79012A06BF02223A71012180F388
:100CCC00118809B10624BDE0FFF78AFC00900120D1
:100CDC0000F0E6F8044610B101203871AFE0FFF7E0
:100CEC00A7FCDFF828180190C1F80090012000F053
:100CFC003FFF012804D1002001F012F94FF0010848
:100D0C00DFF8E047DFF854572168896800208847EE
:100D1C0000F0A1F8687C08B14FF00109287C08B1FB
:100D2C0049F00209E87B08B149F00409E87ADFF8D8
:100D3C00306718B1A16AF08D096B8847A87A18B191
:100D4C00A16A708D096B8847FFF798FF49F0200066
:100D5C00A16A896988470120FFF706FE3878C00729
:100D6C0048BF4FF0010A12D4DFF8980701F03EF9A2
:100D7C008346BBF1040FF7D000F067F880088000C1
:100D8C0008600321A26CDFF87C07526890470020B2
:100D9C0001F034F900F05FF8A06A806B8047BAF17B
:100DAC00000F0AD1A26CDFF85C07526859469047D5
:100DBC0000F04BF840F003000860012021688968BE
:100DCC008847DFF8440700688006FAD5B8F1000FB1
:100DDC001CBF012001F0A4F8A16A49694846884764
:100DEC00A16A496B484688470128F9D1E87A18B1BD
:100DFC00A16AF08DC96A8847A87A18B1A16A708D6A
:100E0C00C96A8847FFF73AFF0020FFF7ADFD0320C2
:100E1C003871042000F044F8DFF8F0160120086067
:100E2C0000F019F801F0F8F9082000F039F8044640
:100E3C00012038710198FFF72BFC01F078F900982C
:100E4C00FFF7D2FB2046BDE8FE8FDFF8D006DFF8B7
:100E5C00CC1600687047DFF8A806006870470000E1
:100E6C0038B58F48DFF878560068EFF3118480F3BB
:100E7C001188E888012803D100F0F0FE0020E880FA
:100E8C0084F3118831BD000010B5FFF759FDEFF365
:100E9C00118481F31188FFF7DFFB84F3118810BDF7
:100EAC0038B500F02AF80844FFF7B2FB002540B92A
:100EBC00204600F008F820B1DFF86806006880478B
:100ECC000225284632BD70B500F017F845182846A3
:100EDC00FFF7A6FB0646B068204206D03169F268DF
:100EEC0020469047C0B2012806D03046FFF7D4FB0D
:100EFC000646AE42EFD1002070BDDFF878150968C8
:100F0C000446DFF8DC05704730BF704770B501F060
:100F1C007FF9DFF840552E6806F00C000C284BD0FA
:100F2C00700727D4FFF7C0FB044600210120FFF710
:100F3C0081FDA0421ED2DFF8C00300680544DFF833
:100F4C0014040668DFF8D8050068B0FBF6F0211A27
:100F5C002846FFF755FB2846FFF756FB4FF47A70EF
:100F6C00B0FBF6F200210120FFF78EFE2846FFF7BA
:100F7C0043FB23E030071FD4DFF8F404DFF8E4442C
:100F8C00DFF87C55F10601685ABF4908490041F069
:100F9C0001010160DFF88405016841F00301016083
:100FAC00202021688969884728682068806B8047E1
:100FBC0001202860286801E0FFF7A6FF01F02CF95A
:100FCC00BDE8704001F0DEB810B50C1801F020F946
:100FDC00401E8041C00FDFF860150A68002AFCD063
:100FEC00246801220A6008B101F016F9204610BDF0
:100FFC0080B50420FFF72AFE0820FFF727FE0E20FD
:10100C00FFF7CEFDDFF82005DFF820150068C0F3F0
:10101C00815003280CBF012000200880DFF8100548
:10102C0002680AB1012002BDDFF8103540221A60B7
:10103C000122C2610020486002BD10B5DFF85C13CC
:10104C00DFF8F04482B009680968202088470F2037
:10105C002060072341F61D5060604FF4C0720220DF
:10106C00009000F0C9F8DFF8D80401210160016894
:10107C008907FCD501212161DFF8B04421880129C1
:10108C0007D1002101610220202100F091F80120FC
:10109C0004E00121002000F08BF80220606013BDF9
:1010AC001C8E00002DE9F041DFF89804DFF87C4439
:1010BC0082B0016842688A4342600161606800281E
:1010CC0004BFBDE8F341FFF7B8BF0128DFF878147F
:1010DC001AD10220606008684BF2F5214843618800
:1010EC00000A11B10021618006E0DFF86014096884
:1010FC0021F07F4108184008DFF854140860000CF8
:10110C004860012088600CE002280FD10868B0F517
:10111C00C06F02D10020606045E00321616000F0E7
:10112C006FF80121BDE8FC41002041E003283DD1CE
:10113C00002060600868A0F5C065A06800F0B2F8F7
:10114C000646284600F0AEF886422CDAA6692846F8
:10115C0000F0ACF88019A061E56860697B4E8542AF
:10116C000ED0A769A7F1100000F09CF8804620690A
:10117C00103800F097F8804502DABFB200970BE008
:10118C00ADB2009508234FF47F423021304600F079
:10119C0094FC206980B2009012234FF4F8020421D1
:1011AC00304600F08AFCBDE8F3418AE0BDE8F381EB
:1011BC0070B50D46DFF89C4382B0032121600021FD
:1011CC00DFF89463316031688907FCD480B20090F9
:1011DC000523602200F010F8012030603068800791
:1011EC00FCD5A561002020600821DFF85003C16008
:1011FC0001600120206073BD0021544800F05DBCEB
:10120C0070B50646514C82B030212046FFF7DCFE0B
:10121C00DFF81853C0F30720E86004212046FFF7DD
:10122C00D3FEC0F384402861A6F5C060A8602E6987
:10123C0000F03CF88019A861A969E868022909DA6C
:10124C00401E6FF03F039842B8BF184610310BD5C3
:10125C00002109E01E2908DB401C4028A8BF3F20C4
:10126C0010392029A8BF1F21A9616861082380B209
:10127C0000904FF47F42302100F011F801200090D3
:10128C0011234FF4003200F009F8A86980B20090E5
:10129C0012234FF4F80200F001F873BD042120462C
:1012AC0000F00BBC002848BF4042704700284CBFE0
:1012BC006FF00101022101EB4000032190FBF1F0E2
:1012CC00704780B5DFF8780200210160016889075A
:1012DC00FCD40021016041600120DFF85412086049
:1012EC000E20FFF7F1FB0820FFF7CEFBBDE8024014
:1012FC000420FFF7C9BB0000008E000010B50446A7
:10130C000020D4E90A2347F6906100F08DFF0123F9
:10131C00994228BF4FF0FF3010BD10B50C4600F0BD
:10132C00FBFF011D201AB0F1004F05D8081BB0F1CE
:10133C00004F38BF8C4200D20C46DFF820221268D6
:10134C00526A2146BDE810400120104700A00C4015
:10135C00048E0000208E0000373F00200440034024
:10136C00401009402DE9F04180460A46D8E90A01AF
:10137C00D8E90C45A0FB026701FB0277A6196F4167
:10138C00340C002244EA07414046FFF7C6FFC8E987
:10139C000E67BDE8F0814FF0FF3002BDA0010010D8
:1013AC00108E0000F8B50546DFF8B801DFF8B8611B
:1013BC000068DFF8B871EFF3118480F3118830689E
:1013CC0040F0800030600120B96849688847F96AAC
:1013DC00096A142088472869BA68526AB0F5802FC8
:1013EC0034BF0421010C012090473A681268232174
:1013FC0000209047B968C96901208847306820F4FB
:10140C00E02040F480303060306840F00100306003
:10141C0084F31188F1BD0000EC3E0020DFF854018C
:10142C0003684068002200211018594170470000E1
:10143C000C200840DFF82411DFF8240110B50968EE
:10144C0044684968012088476069A169BDE810407B
:10145C0008470000B8050020A0860100583E002077
:10146C0054F60100B801001028200860282008401C
:10147C008C210840088E0000148E0000F8B504463C
:10148C000D46FFF7CBFFD4E90A6732463B4600F026
:10149C00CBFE3DB1A6FB002306FB013307FB00335B
:1014AC00C4E90C23F2BD38B5DFF8BC40DFF8C050FE
:1014BC002068400840002060206840F080002060D8
:1014CC000120E062E06A2968496801208847696A5E
:1014DC00096A14208847E06A31BD000030090020F9
:1014EC00B80500209001001080B500F004F8000C45
:1014FC0040EA014002BDDFF8800000688EE7000082
:10150C002C20094000400340141009400C400940B5
:10151C0009B9DFF86810FFF78FB8000024220840E3
:10152C00188E00000C8E0000B43F00506C08002098
:10153C0004800C400C400C4000800C402C500C40A3
:10154C0034600C4028500C4008400C4010200940DE
:10155C003C600C4000400C4038600C408C0100108A
:10156C00E40100201C8E00000020094084010010C2
:10157C008C01001008200940EC010020A0010000A3
:10158C00FEE7704710B5DFF86404046814F1010F2E
:10159C0008BF002400F034FFDFF85414002008606A
:1015AC000120DFF850140860DFF84C140860DFF8F5
:1015BC004C04006828B1DFF848040068204600F0AD
:1015CC0023F8DFF84004DFF840240168890889001B
:1015DC0041F0005141F005010160DFF83004016871
:1015EC006FF31B4111430160DFF824040168C1F360
:1015FC000131012907D10168DFF81824114041F4A9
:10160C0000320260016010BD2DE9F84F0446DFF88E
:10161C00081401200860DFF8040401680029FCD0DC
:10162C00DFF8FC53DFF8FC83C0202860D8F80CA04E
:10163C00D8F80810DFF8F00389075DBFD8F804105C
:10164C00090C41F0F00172210170DFF8E013096818
:10165C00D8F80C20C1F304611629A8BF203901EB7E
:10166C002271491C6FF009029142B8BF114601F07A
:10167C001F0141F4F8510183CAF3C061DFF8B003D4
:10168C0081F001010160CAF3806181F00101816088
:10169C0014B9DFF8A0732DE0DFF89C030068C0F3E9
:1016AC0083615FEA8A32C0F38F2021D44FEA0A4269
:1016BC0012160AD54FF6FF73400804D11846490894
:1016CC0004BF01210120521CF6D4012A10DB40007A
:1016DC0040F00100B0F5803F21BF0120490041F0EE
:1016EC000101102924BF0F214FF6FF70521EECE7A9
:1016FC0040EA014700F08CFD401E8041C00FCF4EE8
:10170C0031680029FCD0DFF83893C9F8107001213A
:10171C00316008B100F080FD0CB9D82008E0C64A51
:10172C0010681168C0F3870001F0030140EA012042
:10173C00009040F2FF3700233A462C21C14800F0BC
:10174C00BCF91CB1BC48C06A8704BF0C00F060FD3A
:10175C00401E8041C00F31680029FCD0C9F81470BC
:10176C000121316008B100F057FD002C0FBFB64FBE
:10177C00B148406A20F0033700F04AFD401E80411A
:10178C00C00F31680029FCD0C9F80C700121316000
:10179C0008B100F041FD0CB9AC4F04E0A648AC49CF
:1017AC00006A01EA000700F033FD401E8041C00FC3
:1017BC0031680029FCD0C9F808700121316008B1EA
:1017CC0000F02AFD0CB9A34F20E09B48806AD8F8A2
:1017DC000830DB07C0F30352C0F303410BD4D8F835
:1017EC0004301F0502EB27721B0482F3040201EB89
:1017FC00237181F30401090441EA025182B242EAE5
:10180C000107222C24BF00F08040074300F000FDAC
:10181C00401E8041C00F31680029FCD0C9F804700B
:10182C000121316008B100F0F7FC2220222C824FFC
:10183C0006D3F86B000F00F00100400040F02000D0
:10184C00854908721120222C05D3F86B400F00F04B
:10185C00010040F01000202C08724FF0000B07D351
:10186C00B86CC10C01F44071C0F3845040EA010B18
:10187C0000F0CEFC401E8041C00F31680029FCD026
:10188C00C9F820B00121316008B100F0C5FC60201E
:10189C00202C06D3B86C000D00F00300400040F083
:1018AC0060006D49C8728020222C06D3F86BC00EE4
:1018BC0000F00100C00040F080000870222C4FF4B2
:1018CC007C4006D3F86B400D00F03F00800040F4E4
:1018DC007C406249DFF888B10880202C0AD3B86CB0
:1018EC000203810A02F47C1242EA815100F00F00DB
:1018FC0041EA003B00F08CFC401E8041C00F316877
:10190C000029FCD0C9F800B00121316008B100F009
:10191C0083FC544844210170882181700CB930211A
:10192C0005E0F96BC90C01F0030141F03001C17005
:10193C004FEA9A5010F0030003D002283CD012D387
:10194C003CE00121042000F0F1F843F2BD70E863A3
:10195C008620286401206864434801680029FCD073
:10196C00002068642EE0012000F002F904462146B4
:10197C00042000F0DBF8042000F0FAF8A042FAD1C1
:10198C00D8F800301802000A81B2E963000C286410
:10199C0001206864344801680029FCD00020686488
:1019AC004FF06022180E314B1B681B6807219847BB
:1019BC004FF48060C9F83800032100E002210420B4
:1019CC0000F0B4F8F8692A4900F03F00087047F6B7
:1019DC001800284908801049274800680020286012
:1019EC000860012025490860BDE8F18F1C130050E8
:1019FC00840460425C600C4008220443800128434C
:101A0C0000012043044003400000390148200340FA
:101A1C0004000940FFFFFCFC101009409402224313
:101A2C0000600C40A83F005056620840B8120050AD
:101A3C0000002043FF0F0F005013005000800C409B
:101A4C0008A00C4000A00C40000088688A76680052
:101A5C00FFFFFC00273F710041A10C40DCA10C40B2
:101A6C0000803F4005A10C4084088C43B401001059
:101A7C000BB00C4070B00C402C2009409404604218
:101A8C0038B504460D4600F0C3FB401E8041C00F24
:101A9C001A490A68002AFCD0012D02D0022D02D06E
:101AAC0003E0247802E0248800E0246801220A6024
:101ABC0008B100F0B1FB204632BD38B500EB410057
:101ACC00102B00F5007402D3103B241D120C04984B
:101ADC00984040EA024500F09BFB401E8041C00F3D
:101AEC0006490A68002AFCD0256001220A600028F9
:101AFC001CBFBDE8314000F08FBB31BD00800C40F5
:101B0C0038B51D460818102D144602D3103D801C04
:101B1C00240C0221FFF7B4FF04EA000188B2E8406C
:101B2C0032BD0268531C03601170704738B504460F
:101B3C00E0070D4607D5A8B2009000230122002132
:101B4C006B48FFF7BAFFA00707D5A8B20090012396
:101B5C00022200216648FFF7B0FF600707D5ADB23F
:101B6C00009502230C2200216148FFF7A6FF31BD2E
:101B7C000146042907BF1D234FF0C0421C234FF020
:101B8C0080525B483421FFF7BBBF10B5594C21681C
:101B9C00896801208847584801688906FCD5216965
:101BAC0009684020884721698968402088471128A6
:101BBC00F9D110BD70B5054600F0AEFB4F4C616815
:101BCC00401A4FF47A714843060C00F023FC21694B
:101BDC00401A48BF4042711940F6B932914207D2BF
:101BEC00062805DAA068E168814201D3226852B95F
:101BFC0043494A68D2074FF4FA6016D40868C0B259
:101C0C007D21484308E0081A3E494843000C00EB8C
:101C1C009000904238BF1046C82801D2C82070BD31
:101C2C00B0F57A6F88BF4FF47A6070BD10B582B092
:101C3C000120009000232E4C012219462046FFF76C
:101C4C003CFF012000900346022200212046FFF7B2
:101C5C0034FF00F061FB2949886013BD80B5012079
:101C6C00FFF786FF01281AD00023012234212048D7
:101C7C00FFF746FFA0B124480068804700F04CFBFA
:101C8C001E498B680A68C860A2EB9202C01A1D4BF1
:101C9C005843000C0860904238BF10460860012081
:101CAC0002BD10B582B0002000900146104C0023FC
:101CBC0001222046FFF701FF00200090014601237E
:101CCC0002222046FFF7F9FE1C234FF080523421EC
:101CDC002046FFF715FF10B10B4800688047074CF2
:101CEC0000F01AFB606000F095FB206113BD000052
:101CFC0000A00C4090010010141009406C3E002014
:101D0C00AC3F005040420F0080000010DFF800F0A4
:101D1C0049C10110DFF800F019C20110DFF800F022
:101D2C0095B70110DFF800F00DC30110DFF800F0DB
:101D3C0081C60110DFF800F08DC20110DFF800F051
:101D4C003DC20110DFF800F009C30110DFF800F00C
:101D5C0045C00110DFF800F0D1C70110DFF800F02A
:101D6C0067BE0110DFF800F021B30110DFF800F0BE
:101D7C0011C80110DFF800F021C80110DFF800F0E5
:101D8C0039C601100C2811D0192814D01D2817D0D1
:101D9C0020281AD021281DD0252820D02A2823D04D
:101DAC002B2826D02C2829D000207047DFF80C02D5
:101DBC00006800687047DFF80402006840687047EC
:101DCC00DFF8F801006880687047DFF8F001006800
:101DDC00C0687047DFF8E401006800697047DFF8FD
:101DEC00DC01006840697047DFF8D0010068C06909
:101DFC007047DFF8C8010068006A7047DFF8BC0163
:101E0C000068406A704700B58BB00A216846FFF73E
:101E1C0089FF0BB000BD00B581B0FEF797FDDFF870
:101E2C00A001DFF8A0110068884218BF00F032F85A
:101E3C00DFF89401B0F5B26F03D001B05DF804EB9C
:101E4C0029E001B000BD00B581B00FF21D00FFF715
:101E5C006DFFFFF763FFFFF76DFFFFF76FFF01B03B
:101E6C005DF804EBFFF76EBF00B581B0FEF7E0FB49
:101E7C00FEF7B6FB01B05DF804EB0320FFF766BF7D
:101E8C0010B504460320FFF761FF2046BDE8104063
:101E9C00FFF760BFFEE7FEE700B581B0FFF75EFF1E
:101EAC00DFF82801C06801B05DF804EBFFF75ABFFA
:101EBC00DFF81C11DFF81C0188617047DFF818117E
:101ECC0001280CBF40F2FF70002008600020704712
:101EDC0030B581B0FFF71AFFDFF800510446E888EF
:101EEC0020B1FFF7BBFE60B10020E880FFF780F85F
:101EFC0005461020FEF7D4FF012D0BD1FFF79DF8FE
:101F0C0008E0052105F13000FEF77AFB05F1300001
:101F1C00FEF77AFB204601B0BDE83040FFF7FABE71
:101F2C0010B5012818D1FFF723FE012816D0FFF7B2
:101F3C007DFEDFF8A8400120E08004F13000FEF7C0
:101F4C005BFB052104F13000FEF75AFB04F1300075
:101F5C00FEF75AFB002010BDFFF7A3FE002010BDBA
:101F6C0010B501240E2805D10120FFF701FE012830
:101F7C0005D003E0DFF86810085C00B900242046A7
:101F8C0010BD00207047FFF7F1BEFFF7F3BE01B99B
:101F9C001449FEF751BB10B588B0044600200190DF
:101FAC000B461820009002AA21460F48FFF7E6FEC8
:101FBC0002A92046FEF7DFFB08B010BDF00100209F
:101FCC0098CA011070472820900500007801002065
:101FDC00440100200004000000000460B80500204B
:101FEC00583E00202C8C00006CF8010000680107A2
:101FFC0001D50420704700F003007047F8B5054682
:10200C007748784C0068800705D50820A071764980
:10201C0076480860F1BD00F0FDF9754A12680021A0
:10202C0012F0030F18BF0121520748BF41F0020103
:10203C000DB141F0040194F90720821A052A02DA45
:10204C00A279914259D0A0F10F0200250023002A59
:10205C001FD402EB02121312082B28BF07231D46B4
:10206C00072D28BF0625634E06EB850756F825502D
:10207C007F687E1BF5B24F0744BFC6F307277D1957
:10208C008F0744BFC6F307477D19CF0748BF05EB41
:10209C001665584E56F82370FEB25FEA417C44BF79
:1020AC00C7F3072C66445FEA817C44BFC7F3074C37
:1020BC0066445FEAC17C48BF06EB1766A2EB0322BD
:1020CC006A434D4B1D681B68A1718032092A9241ED
:1020DC002D17C5F108053427D243DBB27D436B4382
:1020EC0006EBD272B3FBF2F2B2F5803F28BF4FF68B
:1020FC00FF7200F30700A280E07140480068A188DD
:10210C00206000201F2904D21F21A18004E049086F
:10211C00401CB1F5007FFAD20F39090940EAC10021
:10212C00314A37490843106000205060F1BD10B5AA
:10213C003448006884B224B300F06CF9294991F951
:10214C000720904205DA6FF07F029042B8BF10462C
:10215C00C8718888844201D28C8010BD274A1268CD
:10216C000B68D21A921C202A28BF1F22231A52084D
:10217C0023FA02F42018B0F5803F28BF4FF6FF7009
:10218C00888010BD2048006800B9704710B41F4902
:10219C008A6802F04063B3F1406F1ED04B689B0716
:1021AC001BD40F4B1C680968C1F303511C31090186
:1021BC0014F0050F06D088420FD224F005001860E9
:1021CC0010BC7047814208D2100158BF44F0010482
:1021DC00500158BF44F004041C6010BC7047000050
:1021EC0000000940F43E002030100940FDFDA40021
:1021FC00242208409C130050B43F00500820094092
:10220C0000FFA4803410094028500940AC3F005016
:10221C00EFF3108072B67047EFF3108062B6704720
:10222C000138FDD1704770471B4213D1094236D19A
:10223C002AB18446B0FBF2F002FB10C2704700F0EA
:10224C00FDB8FCD30022002370470B0002000021D4
:10225C0000207047904271EB030CF6D370B5B1FAC5
:10226C0081F4B3FA83F52C1BA340C4F1200532FA98
:10227C0005F63343A2405FF00046E64002E05B08FF
:10228C005FEA3202841A71EB030524BF204629460B
:10229C007641F4D302000B003000002170BD012AFE
:1022AC00CFD970B5140C20D0B1FA81F4B2FA82F502
:1022BC00C4F120046419B4F12006D6D3B2405FF007
:1022CC000044F440002502E052085FEA3303C61ACA
:1022DC0071EB020E24BF3046714664416D41F3D35D
:1022EC0002000B002000290070BD0C46B1FBF2F17E
:1022FC0002FB11452D0445EA1045B5FBF2F402FB37
:10230C00145580B240EA0545B5FBF2F002FB1052C1
:10231C0040EA044070BD000038B5FFF779FF06496C
:10232C000C684D68401E8041C00F18BFFFF774FF4A
:10233C00280C40EA044032BD082009402D480068B2
:10234C00000C00F00700032828BF4FF0FF30704747
:10235C0029490968C1F30F314BF69A1291424FF09B
:10236C00FF3001D1002070474BF6BE12914201D1D3
:10237C00012070474BF62032914208BF0220704773
:10238C0010B41D491D4B0A681B680968120FDBB29B
:10239C00802B28BF0023C1F30F314BF69A14A142B6
:1023AC004FF0FF300CD1012A08D0032A1DD0072A88
:1023BC001DD0082A08BF03F1160013E00A2011E013
:1023CC004BF6BE14A14206D1002AF7D0022A09D13D
:1023DC0003F1140006E04BF62034A14204BF002A9E
:1023EC0003F10A0010BC40B270471420FAE7152024
:1023FC00F8E700009412005018130050A010005081
:10240C0080B5FFF7A5FF18B9FFF7BAFF162800DA59
:10241C00FEE701BD0748084A816812780068C903C5
:10242C0052B2A0F54070C9135043A1EB201080307C
:10243C0000127047285009400C13005070470000E0
:10244C002DE9F04FA1B08246002016461D460291A0
:10245C000B900DF144086FF000490AE016F8011BCF
:10246C000298D0470028029000F0B9820B98401CCB
:10247C000B903078010001D10B98B2E22528EDD1F8
:10248C000020059006900790089009900A9001E0B2
:10249C0040F0010016F8011F2029F9D023290DD096
:1024AC002B2904D02D2906D030290AD00CE040F07D
:1024BC00020080B2EEE740F00400FAE740F00800BA
:1024CC00F7E740F01000F4E72A290ED129682960BB
:1024DC0051F8042B2960002A0D9204D5514240F08A
:1024EC0004000D9180B2761C11E000210D9109E0E1
:1024FC000D99494505D001EB810302EB43013039BD
:10250C000D91761C3278A2F130010A29F0D3317882
:10251C002E2903D04FF0FF310C911DE016F8011F4E
:10252C002A2907D129682960761C51F8042B2960C7
:10253C000C9211E000210C9109E00C99494505D051
:10254C0001EB810302EB430130390C91761C32789C
:10255C00A2F130010A29F0D3ADF838000FF6A840EB
:10256C00317800F05FFE08B116F8010B8DF83A00D7
:10257C009DF83A00682802BF31786829622005D09E
:10258C006C2804BF30786C2803D171208DF83A0088
:10259C00761C11A8049016F8017BB7F125002AD0FF
:1025AC001C3800F0CA80001F022840F2C680133885
:1025BC0000F0ED80093800F0C080801E00F05A81D8
:1025CC00401E00F03081401E022840F2B680001FF1
:1025DC0000F02981401F00F08180401E00F0D78060
:1025EC00401E24D0C01E0BD0801E00F0D080C01E18
:1025FC0000F0CD8048E125208DF8440001204DE10C
:10260C002868286050F8044B286003940C9F002F16
:10261C0004D5204600F012FE074606E03A4600219B
:10262C00204600F027FE00B1071B069737E129680A
:10263C002960002251F8040B29600021CDE900012A
:10264C0011A80390DDE900019142049F08BF90425C
:10265C004FF03C0C01D10C9AC2B100F00F03303397
:10266C00DBB23A2BA8BF2733ACF101020009BB54F3
:10267C00944640EA017009090022914208BF904239
:10268C0004D0039A07EB0C039A42E6D307EB0C0039
:10269C000390CCF13C010C980691814209DA401A66
:1026AC0008904FF6EF71BDF838000840ADF83800CF
:1026BC00F5E0002840F1F3809DF8380000F014009C
:1026CC00102840F0EC800D98059A801A089A801A10
:1026DC00401A0128C0F2E3800890E0E09DF83A002F
:1026EC0062281AD0682806D06A280CD06C281CD016
:1026FC00712808D019E02868286050F8041B28605D
:10270C000B980880CBE02868286050F8042B2860D0
:10271C000B98C117C2E90001C1E02868286050F885
:10272C00041B28600B980870B9E02868286050F8E2
:10273C00041B28600B980860B1E02868C01D6FF07E
:10274C00070101EA00022A60D2E9000108322A607E
:10275C00CDE90001002902D505982D210AE0BDF82C
:10276C003800810702D505982B2103E0C00705D559
:10277C000598202108F80010401C059011A8059917
:10278C00084403903946684600F0ECF987E09DF860
:10279C003A006C280FD0712818BF6A280BD1286812
:1027AC00C01D6FF0070101EA00022A60D2E90001A6
:1027BC0008322A6005E02968296051F8040B296069
:1027CC000021CDE900019DF83A00682803D1DDE92C
:1027DC00000180B20BE0622803D1DDE90001C0B238
:1027EC0005E0742818BF7A2804D1DDE90001002126
:1027FC00CDE900019DF83800000732D5DDE9002352
:10280C000020834208BF82422BD047F0200078285A
:10281C0027D10598302108F80010401C411C059167
:10282C0008F800701DE09DF83A00294600F0DCF82D
:10283C00CDE90001DDE9002300218B4202DA059885
:10284C002D210AE0BDF83800810702D505982B210F
:10285C0003E0C00705D50598202108F80010401C9E
:10286C00059011A80599084403903946684600F074
:10287C00F3F814E0012005902868286050F8041B38
:10288C0028608DF844100AE025208DF844000120C2
:10289C000590380003D088F80170022005900D983F
:1028AC000599401A0899401A0699401A0999401A34
:1028BC000799401A0A99471A9DF83800400710D416
:1028CC002020012F8DF840000BDB3C46012310AA81
:1028DC006946504600F081FC002840F08080641E60
:1028EC00F4D1DDF814B0BBF1000F11AC0CD014F81E
:1028FC00011B0298D0470028029070D00B98401C06
:10290C00BBF1010B0B90F2D130208DF84000089CEC
:10291C00012C09DB012310AA6946504600F05DFC2E
:10292C0000285CD1641EF5D1DDF818B0039CBBF116
:10293C00000F0CD014F8011B0298D047002802900D
:10294C004DD00B98401CBBF1010B0B90F2D13020F9
:10295C008DF84000099C012C09DB012310AA694663
:10296C00504600F03AFC002839D1641EF5D103988A
:10297C000699DDF81CB04418BBF1000F0BD014F80D
:10298C00011B0298D047029048B30B98401CBBF136
:10299C00010B0B90F3D130208DF840000A9C012CD8
:1029AC0008DB012310AA6946504600F016FCB0B9AA
:1029BC00641EF6D19DF8380040077FF55AAD2020F3
:1029CC00012F8DF84000FFF654AD012310AA694683
:1029DC00504600F002FC10B97F1EF6D149E54FF0CD
:1029EC00FF3021B0BDE8F08F622827D068281ED0B8
:1029FC006A2808D06C2828D0712804D0742824D0D8
:102A0C007A280DD021E00868C01D6FF00702104035
:102A1C000860D0E90023083008601946104670475A
:102A2C000A680A6052F8040B0A60002170470A68B1
:102A3C000A6052F8040B0A6000B20BE00A680A60E4
:102A4C0052F8040B0A6040B204E00A680A6052F8BB
:102A5C00040B0A60C11770472DE9F343054608467D
:102A6C002F696F2808BF082405D041F02001782970
:102A7C0014BF0A2410243C26D5E90023642818BF6F
:102A8C0069289046994606D100218B4203DAD8F189
:102A9C00000869EB49090020814508BF80450CD12D
:102AAC00286B50B9082C38D195F83800000734D56C
:102ABC0030203B2687F83B002FE0701E0090064626
:102ACC00404649462246E317FFF7AEFB02F13000C1
:102ADC00C0B23A2803DB9DF8041051390818B855D8
:102AEC00494640462246E317FFF79EFB804689463F
:102AFC000020814508BF804503D0E868B919884299
:102B0C00DBD3082C09D195F83800000705D5B85D42
:102B1C00302802D0761E3020B855B919E960C6F1BC
:102B2C003C00296BA861884208DA081A28624FF623
:102B3C00EF71288F08402887BDE8F38300290ED554
:102B4C0095F8381001F01401102908D1696B6A69E5
:102B5C00891A2A6A891A0E1A012EA8BF2E62BDE89C
:102B6C00F38300002DE9F24F04468EB0D4E9000146
:102B7C00CDE9020104AF9DF8380040F0200BBBF109
:102B8C00610F0AD0206B002848BF062004D408BF70
:102B9C00BBF1670F01D1012020636168C1F30A50BA
:102BAC0040F2FF7290421CD1080304BF2068002839
:102BBC0009D10320A0619DF8380061381A2835D35B
:102BCC000FF2586108E00320A0619DF838006138CD
:102BDC001A2828D30FF23C61E068032200F076FB40
:102BEC00C3E1012815DA204600F0ABFB012810DB0D
:102BFC0000250020BBF1610F1FD1E16830220A7063
:102C0C008A1CE2609DF83820612A0CBF7822582279
:102C1C000FE0626840F2FE3161F31E52451A6260A9
:102C2C004FF0FF30E6E70FF2E851D5E70FF2E8512D
:102C3C00D2E74A706169891C616110B900260025D0
:102C4C008AE1BBF1610F40F09880206BD4E900ABB6
:102C5C0000284CBF2126461CDDE90201002200237E
:102C6C0000F092FB36B23ABF8BF00040CDE902A0E7
:102C7C00CDE902AB06F101082D1FB8F1010F8DF85B
:102C8C0010200DF1110736DBDDE9020100220023D3
:102C9C0000F092FB2FD21C2102A800F0A5FBDDE96D
:102CAC00020100F027FCA8F10708B8F1010F8146DA
:102CBC0009DB00F04BFC02460B46DDE9020100F09B
:102CCC005DFCCDE90201F81D072105E009F00F02BA
:102CDC0000F8012D4FEA2919B9F1010F01DB491E4A
:102CEC00F4D5491E5CBF002200F8012DF9D5C71D93
:102CFC00B8F1010FC8DA0DF11100391AB142B8BFA1
:102D0C000E4636B230000DF111072FD4884206DA88
:102D1C0004A9014449780829A8BF0F2100DA002131
:102D2C0004AA024400E0761E12F80139401E8B42C0
:102D3C00F9D00F2904D104A901444A78521C4A70D5
:102D4C00002802D504AF761C2D1D36B2701E0DD492
:102D5C0039180A783032D2B23A2A03DB9DF838306F
:102D6C003A3B9A18401E01F80129F2D5206B002835
:102D7C0040F1F280701E2063EEE0DDE902010022DA
:102D8C00002300F001FB3CBF81F00041CDE90201C2
:102D9C002DB247F2975068434D49DFF8389180FBCC
:102DAC0001214D1305EBD5752DB2C5F1070ABAF10A
:102DBC00010F98461CDBDDE902675FEACA7007D594
:102DCC0042464B463046394600F098FC06460F46C4
:102DDC004046494642464B464FEA6A0A00F08EFC92
:102DEC00BAF1000F80468946E7D1CDE9026724E0AD
:102DFC00CAF1000A0026384F14E05FEACA7007D502
:102E0C0042464B463046394600F078FC06460F46A3
:102E1C004046494642464B4600F070FC4FEA6A0A6F
:102E2C0080468946BAF1000FE7D1DDE9020132464E
:102E3C003B4600F035FDCDE90201BBF1660F216B7D
:102E4C00DFF898900CBF05F10A0006204618142EE6
:102E5C00A8BF132630208DF810000DF11107012E9C
:102E6C0040DBDDE9020100F05BFB07F10801042205
:102E7C001B4FA0FB0773DB0803EB8307A0EB47009A
:102E8C00303001F8010C164FA3FB0770C00800EBA3
:102E9C008007A3EB47033033521E01F8023DE7D104
:102EAC00083E012E01F10807D9DBDDE9020100F033
:102EBC0037FB00F055FB02460B46DDE9020100F042
:102ECC005DFB00224B4600F019FCCDE90201C8E77E
:102EDC0089B5F814000024400000F03F84D79741D6
:102EEC00CDCCCCCC0DF11100381A0DF1110702E04C
:102EFC00401E6D1E7F1C39783029F9D0BBF1660F4E
:102F0C0008BF691C04D0BBF1650F0CBF0121002167
:102F1C00226B8E1836B2B042B8BF064636B23100BC
:102F2C001AD4814204DA785C3528A8BF392000DA3B
:102F3C0030207A18521E00E0761E12F80139491E14
:102F4C008342F9D0392802D1785C401C785400298E
:102F5C0002D57F1E761C6D1C2DB29DF83810009585
:102F6C0033B23A46204600F003F80FB0BDE8F08FBC
:102F7C002DE9F043054685B01F46D5F83080012F6A
:102F8C008946164602DA01270FF2942649F02000F2
:102F9C00BDF93040662808BF641C17D0672840F084
:102FAC00848014F1040FC0F28680444580F2838043
:102FBC0095F83800641C000702D44745B8BFB846E2
:102FCC0024B2B8EB040848BF4FF0000824B2E868FC
:102FDC00A969012C27DA4A1C30234354B8F1010F9C
:102FEC0003DA95F83800000703D5E9682E208854D9
:102FFC00521C18EB040FB8BFC8F1000424B2604295
:10300C006862A044B845AA61B8BF4746E868AB6996
:10301C003FB2EF613A463146184400F057F9A8EB3D
:10302C000700A862C2E022469742084418DA3A46E2
:10303C00314600F04BF9A9697918E01BB8F1010F82
:10304C00A961686203DA95F83800000705D5EA68CB
:10305C002E205054E869401CE861C5F82880A5E092
:10306C00314600F033F9A86920183F1BB8F1010F65
:10307C0003DA95F83810090703D5EA682E211154A4
:10308C00401CA8613FB2B845B8BF4746E868AB6979
:10309C003FB23A463119184400F018F9A8693818AB
:1030AC00A861A8EB0700686280E0B9F1610F16D146
:1030BC004FF0700918E0474504DA95F83810090705
:1030CC0058BFB846B8F1010848BF4FF00008B9F135
:1030DC00670F14BF4FF045094FF0650904E0B9F1D3
:1030EC00410F08BF4FF05009A969EB68481CA86153
:1030FC00B8F1010F16F8012B5A5403DA95F8381071
:10310C00090719D5EA68431CAB612E211154B8F19B
:10311C00010F11DB7F1E3FB2B845B8BF4746E868C8
:10312C003FB23A463146184400F0D0F8A869381836
:10313C00A861A8EB07006862E868A969014420004F
:10314C0081F8009003D42B2048708E1C03E02D22B4
:10315C004A708E1C644200270DF1080808E00A2210
:10316C00684600F0C8FC019808F8010B7F1C009C15
:10317C0021B20129F3DA022F06DA49F02000652882
:10318C0004BF302006F8010B4FB9302006F8010BB4
:10319C0007E07F1E02A8C05D303006F8010B012F3E
:1031AC00F7DAE868A9690844301AE86195F838003C
:1031BC0000F0140010280DD16869A9690818696A13
:1031CC000818E9690818A96A0818696B8842BCBF15
:1031DC00081A286205B0BDE8F083F8B504460D4620
:1031EC0016461F46002077B116F8011BA868A047A9
:1031FC00A86030B1E86A401CE86200207F1EF3D161
:10320C00F2BD4FF0FF30F2BD686A6C747A4C00006E
:10321C006E616E004E414E00696E6600494E46006E
:10322C00300000000278C9B28A421AB11CBF10F8F3
:10323C00012FF9E718BF00207047000000F10103CF
:10324C00810704D010F8011B89B18107FAD10268FB
:10325C00B2F10131914311F0803F04BF50F8042FBB
:10326C00F6E710F8011B11B110F8011BFBE7C01AAF
:10327C0070470000C9B2830706D0521E22D310F843
:10328C00013B9942F7D11FE0083A13D302F1040233
:10329C0041EA012141EA014150F8043B121F21BFD0
:1032AC004B40A3F1013C2CEA030C1CF0803FF3D003
:1032BC00C9B2001F083210F8013B521E28BF91EA18
:1032CC00030FF8D818BF0120401E704762B38B075C
:1032DC0008D0521E11F8013B00F8013B00F024808D
:1032EC008B07F6D1830740F0208000BF103A07D33C
:1032FC0030B4B1E83810103AA0E83810F9D230BC2C
:10330C00530724BFB1E80810A0E8081044BF51F8D7
:10331C00043B40F8043BD20724BF31F8022B20F8C1
:10332C00022B44BF0B7803707047083A07D3B1E8FF
:10333C000810083A40F8043B40F804CBF7D2530786
:10334C00E4E730B4436803F000420121C3F31303F4
:10335C004360002B04BF0368002B08D10DE0036809
:10336C00DD0F45EA440444605B000360491E446879
:10337C00E302F4D5C4F31303436043681A43426079
:10338C00084630BC704700004FF4001C1CEB410F8A
:10339C0094BF1CEB430F09E041EA030C50EA4C0CC0
:1033AC0052EA0C0C03D2994208BF9042704714BFEA
:1033BC008B428242704700004FF4001C1CEB410F03
:1033CC0094BF1CEB430F09E041EA030C50EA4C0C90
:1033DC0052EA0C0C03D28B4208BF8242704714BFD6
:1033EC00994290427047000070B504460D466068E3
:1033FC00C0F30A5040F2FF71884207D160680003A5
:10340C0004BF2068002817D0022070BD20B92046C8
:10341C00FFF797FF012866DA012D0FDB40F2FF71F1
:10342C00091A8D420AD36068002847BF00202F4933
:10343C0000202F49C4E90001012070BD4142A9427E
:10344C00616806DA6FF31E51401941EA0050606062
:10345C0040E0401E63684519012205F1350062F316
:10346C001F53352801F00041636003D361600020D5
:10347C00206070BD002015F11F0F04DA2068236056
:10348C000022203562606A4212D0401E25688041BD
:10349C00C2F12003C0439D4045EAD07025686668A0
:1034AC00D54006FA03F32B4323606368D340636073
:1034BC0062680A43B0F1004F626003D80DD12078E6
:1034CC00C0070AD52068401C2060206828B96068B5
:1034DC00401C60604FF0FF3070BD6068884204BFD4
:1034EC0020680028F6D1002070BD00BF0000F0FF5E
:1034FC000000F07FF446400D40EAC120490006D29E
:10350C0000F014F8004248BF6FF00040604700F034
:10351C000DF84FF0004188428CBF0846404260478E
:10352C00400D40EAC120490080F00D8040F0004081
:10353C00490DA1F58061491C05D4D1F11F0154BF7F
:10354C00C840C01770474FF000007047010040F1B1
:10355C000980F446404200F005F851F00041604704
:10356C00010000BF09D0B0FA80F18840C91CC1F538
:10357C008461090501EBD02140057047F0B44FF090
:10358C00004591EA030F44BF6B4000F0BBBA00BF8B
:10359C00841A71EB030604D26E40001BB141121960
:1035AC0073414FF4001C1CEB410F34BF7CEB430602
:1035BC0084E00C0DA4EB1356362E7DDC012E43DC7F
:1035CC0045EAC32343EA525312BFD20292025B086C
:1035DC00240545EAC12141EA5051D2EBC020994162
:1035EC0025D407D1B0FA80F610FA06F164D0002089
:1035FC00203608E0B1FA81F6B140C6F1200220FA7B
:10360C0002F21143B0404FEAF474B4EB465434F078
:10361C0001064FEA74040AD8D6F50016760D04F0AC
:10362C000044F04061FA06F25040F1404840C00AB4
:10363C0040EA415021F0004128BF5FEA500550F1AB
:10364C00000044EBD12137E045EAC323DB0A45EA0D
:10365C00C121C90AB6F120050EDD42EA0242120C64
:10366C00C5F1200603FA06F6EB4042EA06056D4268
:10367C00984161F100010DE062FA06F5F240554007
:10368C0063FA06FC82EA0C02F3405A406D42904108
:10369C0061EB030111F4801F05D1641E620502D099
:1036AC006D004041494121F48011430875F10043FC
:1036BC0050F1000041EB0451F0BC70471CEB410F82
:1036CC0015D223F0004352EA43060BD04FEA4C0CC0
:1036DC00BCEB410F04D80C0D661E342EB7DDEBE7A6
:1036EC00801A994150EA410608BF0021E4E708BF5F
:1036FC001CEB430F28BF6FF00001DDE7B0B581EA8A
:10370C00030C0CF0004C40F2FF7515EA11541DBF70
:10371C0015EA1357AC42AF4239E0E41923EA45539A
:10372C0043F48013C90241F0004141EA505EC702E4
:10373C001100A7FB020200284FF00000EEFB012055
:10374C004FF00001E3FB072118BF42F001024018C3
:10375C0000214941E3FB0E01A4F580640F0302D262
:10376C0052004041494154F101046CDD470872F1AB
:10377C00004250F1000051EB0451A1F580115CBFE7
:10378C0041EA0C01B0BD4CEA05510020B0BD05EA80
:10379C001357AC4214BFAF4241E050EA410E1CBF7C
:1037AC0052EA430E02E061460020B0BD24423C4484
:1037BC001BD15FEA070EF6D0090302BF01460020B9
:1037CC00AEF1140EB1FA81F7AEEB070401FA07FE65
:1037DC000C37C7F1200100FA07F7C8404EEA000E7B
:1037EC0023EA455343F48013A2E733F00043B3FAC2
:1037FC0083F704BFB2FA82FE77440B3FE41BB7F1A8
:10380C00200E2FBF02FA0EF3BB40C7F1200E22FA96
:10381C000EFE38BF43EA0E03BA40641C82E750EA3E
:10382C00410E14BF52EA430E6FF000014FF4001723
:10383C0017EB430F8ABF194617EB410FB5E74CEA5C
:10384C0005510020B0BDD4F10104B4F120070FDA0A
:10385C00C4F12007520828BF42F0010210FA07F504
:10386C0001FA07F7E1BF2A43E0403843E1400FE09B
:10387C00352C98DCC7F1200452EA400220FA07F2FA
:10388C0018BF42F0010231FA07F0A1400A430021AF
:10389C0072F1004250F1000051EB0C01B0BD000080
:1038AC002DE9F04140F2FF7581EA030C0CF0004C5D
:1038BC0015EA11541DBF15EA1357AC42AF42E9E0AB
:1038CC00BC41C1F31301C3F31303801A994143F4B0
:1038DC00801304D2641E4000494180185941C9022A
:1038EC0041EA5051B1FBF3F603FB1611A2FB06752E
:1038FC00D7EBC020A94102D2761E80185941C902CB
:10390C0041EA5051B1FBF3FE03FB1E11A2FB0E75F5
:10391C00D7EBC020A94103D2AEF1010E801859415A
:10392C00890241EA9051760546EA8E2EB1FBF3F6F8
:10393C0003FB1611A2FB0675D7EB8020A94102D21E
:10394C00761E80185941C90241EA50514EEA060EC2
:10395C00B1FBF3F603FB1611A2FB0675D7EBC020E7
:10396C00A94102D2761E80185941C90241EA505130
:10397C00B1FBF3F703FB1711A2FB0735D3EBC02008
:10398C00A94167F100070CBF004247F0010766F33D
:10399C00D5274FEA1E31B80814F5806414DDBD0735
:1039AC0075F1004250EB0E5051EB045111F5801F94
:1039BC005CBF41EA0C01BDE8F0814CF07F6141F045
:1039CC00E0410020BDE8F081BD076D0840EA0E50D3
:1039DC0041F48011D4F10104B4F120060ADAC4F1E7
:1039EC0020060200E04001FA06F3E1401843B24021
:1039FC0015430EE0342C14DCC6F1200445EA4005D6
:103A0C006D0820FA06F2154321FA06F0A1400D4389
:103A1C00002175F1004250F1000051EB0C01BDE8A2
:103A2C00F08100205FEA0C01BDE8F081CFB992185B
:103A3C005B41B3FA83F704BFB2FA82F6BF190B3FAE
:103A4C00B7F120062FBF02FA06F3BB40C7F12006E0
:103A5C0022FA06F638BF3343BA401CB1E419641E8F
:103A6C002FE77F4231F00041B1FA81F404BFB0FA84
:103A7C0080F6A4190B3CB4F120062FBF00FA06F116
:103A8C00A140C4F1200620FA06F638BF3143A0400D
:103A9C003C1B16E7AC421ABF05EA1357AF4214E0C1
:103AAC0050EA41061CBF52EA4306BFE750EA410701
:103ABC00304661461CBF41EA0551BDE8F08152EA2F
:103ACC00430C08BFC143BDE8F08100204FF4001641
:103ADC0016EB410F98BF16EB430F08BF16EB410FC7
:103AEC0024BFC14305E016EB430F0CBF61464CEA03
:103AFC000551BDE8F08191FBF2F303FB1211C0E913
:103B0C0000317047841A71EB030603D2001BB141DC
:103B1C00121973414FF4001C1CEB410F34BF7CEBAA
:103B2C00430443E00C0DA4EB1356352E50DC45EA50
:103B3C00C323DB0A45EAC121C912B6F120050DDD0C
:103B4C0063FA05F6EB4086EA0305124218BF45F00E
:103B5C000105C01851F100010CD213E062FA06F510
:103B6C00F2405540F3415A40B340F3405A4080185C
:103B7C00594107D349085FEA30005FEA350528BF91
:103B8C0045F0010501F58011420875F1004250F134
:103B9C00000041EB0451F0BC4FF4001C1CEB410F36
:103BAC0038BF70470020090D090570471CEB410F09
:103BBC0010D252EA43060BD0BCEB410F05D80C0DCA
:103BCC00AB43661E342EB5DD02E0AB438018594181
:103BDC00F0BC7047F0BC7047DFF800F0D9C10110A1
:103BEC00DFF800F041AC0110DFF800F025B1011056
:103BFC0080B5002804D008233C220021FFF7ECFFFD
:103C0C0001BD3EB504000D000820ADF800000120F8
:103C1C00ADF802006846DFF8CC1909688847BDF892
:103C2C0004102180029929603EBD00B583B00821A3
:103C3C00ADF800100321ADF8021001906846DFF8D2
:103C4C00A4190968884707BD70B584B004000D003D
:103C5C0016000820ADF800000920ADF802006846F7
:103C6C00DFF8801909688847BDF804102180BDF879
:103C7C00061029800299316004B070BD00B583B084
:103C8C000821ADF800100A21ADF802100190684629
:103C9C00DFF85019096888470EBDE0B50821ADF86A
:103CAC0000100421ADF8021080B201906846DFF8D4
:103CBC00341909688847002801D0002000E00298D8
:103CCC000EBD00B583B00821ADF800100521ADF88C
:103CDC00021001906846DFF80C190968884707BD87
:103CEC00DFF804090068704730B599B06422694662
:103CFC00822000F0E0FF6846FFF7A0FA0400601C89
:103D0C00DFF8E81808700920DFF8E01848706946F9
:103D1C00DFF8DC5822002800FFF7D8FA0922DFF878
:103D2C00D418DFF8C8082044841C2000FFF7CEFA12
:103D3C0019B030BD00B58FB06846FFF759FFDFF8FA
:103D4C00B808079040F6C410089001200690002394
:103D5C006A460FF20931DFF8A408FFF745FF0FB0F0
:103D6C0000BD10B58EB0DFF89C18DFF89C08FFF78B
:103D7C0048FF00F095FE00208DF80800012202A9F2
:103D8C00882000F098FF9DF8080000280ED00CA8A1
:103D9C00DFF87818D1E90023C0E9002306220CA92A
:103DAC00812000F088FF0CA801F091FCFFF79CFF2C
:103DBC00DFF85C18DFF85C0801F04AFEDFF8401809
:103DCC000860DFF8540801F09EFFDFF85018086017
:103DDC00DFF84C0801F097FFDFF848180860102056
:103DEC00019000200090002364220FF26971DFF82B
:103DFC00380801F03DFF06211F2001F0B8FA012020
:103E0C008DF80E000020ADF81C0001208DF80D007F
:103E1C001020ADF81A001020ADF818000020ADF8F5
:103E2C0016004FF4FA60ADF814000DF10E020121EA
:103E3C0040F2053001F0D4FF07AA022140F206300F
:103E4C0001F0CEFFDFF8A407FFF7F8F90100DFF867
:103E5C009C27C9B24FF4427001F0C2FFDFF8CC27A7
:103E6C00072140F2073001F0BBFF0DF10D020121DB
:103E7C004FF4447001F0B4FF0DF11A02022140F22C
:103E8C00113001F0ADFF06AA022140F2123001F010
:103E9C00A7FF0DF11602022140F2133001F0A0FF32
:103EAC0005AA02214FF4457001F09AFF152100225A
:103EBC00DFF87C47200002F03FFC1522DFF870177A
:103ECC00822000F0F8FEDFF86807FFF7B7F9010071
:103EDC00DFF85C27C9B2002001F04AF92020ADF8C8
:103EEC0012002020ADF8100004220DF112018920DF
:103EFC0000F0E1FE042204A98A2000F0DCFEBDF8EB
:103F0C001210062001F033FABDF81010072001F052
:103F1C002EFABDF81210082001F029FABDF8101085
:103F2C00092001F024FA00200B9001208DF80C00E0
:103F3C0001208DF80B0000208DF80A0001208DF86F
:103F4C0009000BAA04214FF4816001F065FA03AA61
:103F5C0001214FF4806001F05FFA0DF10B02012199
:103F6C0040F2024001F058FA0DF10A02012140F230
:103F7C00034001F051FA0DF10902012140F2064013
:103F8C0001F04AFA5FF0FF3001F0EFF85FF0FF301C
:103F9C0001F0B4F802F004FC5FF0FF3002F00AFD0F
:103FAC00DFF8900602F031FDDFF88C0602F0ECF839
:103FBC00DFF8880601F066F85FF4E1300A90032020
:103FCC0009900020089008AA09A90AA800F05AFB39
:103FDC000A98DFF86C1688610998DFF86416087780
:103FEC000898DFF85C164877DFF8540602F01DFEDF
:103FFC00DFF814060088C0B201F041F8DFF80806BB
:10400C000088C0B201F097F80FF2615002F0A5FFE2
:10401C000FF2595002F0F4FD202001900020009086
:10402C0000234FF47A720FF22D51DFF8180601F0CD
:10403C001FFE0020009001226946862000F03BFE06
:10404C000098002806D0DFF8FC0501F035FE0820AA
:10405C0000F0DAFE0EB010BD0000000010B584B008
:10406C00FFF77FFE8EE0DFF8B405006801F076FE06
:10407C000400002C05D0200000F0C8F92000FFF748
:10408C0020FEDFF898050068FCF7C2FA0028EAD099
:10409C00DFF8B405007840070AD5DFF8AC050088D6
:1040AC004FF6FB710840DFF8A015088000F051FABC
:1040BC00DFF894050078800664D5DFF8900502F0EF
:1040CC0087FFDFF8840500884FF6DF710840DFF8C2
:1040DC0078150880DFF87805007806284ED0DFF8D0
:1040EC0070050078072849D0FDF718FEDFF8640545
:1040FC0002F06EFF0120DFF86015096849688847F7
:10410C0046F2CE410120DFF850251268526A9047E2
:10411C00FFF7E6FDDFF84405FEF782F80420FCF714
:10412C00B3FC0820FCF7B0FC002200210120FCF7B6
:10413C00ABFD0420FCF78AFD0820FCF787FDDFF8B7
:10414C001C05FEF76DF80620FCF770FC0920FCF747
:10415C006DFC01208DF8040001AA012140F205300C
:10416C0001F03EFEDFF8D80402F05FFD4FF4FA5088
:10417C00FEF756F8DFF8E80402F02AFFDFF8E40453
:10418C0002F026FF5FF0FF30FFF778FD00287FF488
:10419C007FAF002000906A4602A90DF10600FFF7E0
:1041AC0053FD002824D10124BDF80600102816D197
:1041BC00BDF80800DFF85014098888420FD1009828
:1041CC0001884FF6FF72914205D18078000706D521
:1041DC0000F0D6F803E0009800F0A2F80400009874
:1041EC00002805D0E4B2002C02D00098FFF71DFD8A
:1041FC00DFF830040068FCF70BFA00287FF441AFBD
:10420C00DFF820040068FCF70BFA8468002C3FF4FC
:10421C0038AFDFF854040078012857D1DFF83004A8
:10422C000078062804D0DFF82804007807284DD140
:10423C000120207810280ED0202846D1601CC0B256
:10424C0002F01EFCDFF8DC03006801F087FD2000A3
:10425C00FFF737FD15E7627DDFF81014601C02F0E4
:10426C00FFFE002808D10020DFF8FC1308700020A6
:10427C0000F0CAFD002004E0621C617D002002F009
:10428C00CBFBC0B2002807D0012002F0FFFEDFF804
:10429C00E00301F011FD17E0607D80B202F0E5FB58
:1042AC00DFF88003006801F059FDDFF8780300683F
:1042BC00FCF7AEF9002804D1DFF848030068FFF7DB
:1042CC008FFC2000FFF7FDFCDBE6DAE6627DDFF811
:1042DC009C13601C02F0C4FE002807D10020DFF8FC
:1042EC0088130870002000F08FFD03E0617D601CD6
:1042FC0000F064FA607D80B202F0B7FBC948006838
:10430C0001F02CFDC7480068FCF782F9002803D1A6
:10431C00BC480068FFF764FC2000FFF7D2FCB0E655
:10432C0080B5010001200A78912A05D0B02A07D166
:10433C00080000F007F803E049780E29FFD0FFE7EA
:10434C00C0B202BD10B50400607816280FD1082247
:10435C00AD480188C9B2608801F0C1F9002808D1C4
:10436C00012000F038F8C3480460002007E02079F1
:10437C007E28217914F1080001F09CF8012010BD71
:10438C0010B5BC480068002824D0BB480078401CFD
:10439C00B9490870B748006810F10802B5480068C0
:1043AC000179B4480068408800F0CDFE0400E4B206
:1043BC00162C0FD0E4B2042C0CD0002292480188A9
:1043CC00C9B2AC480068408801F089F92000C0B23D
:1043DC0000F001F810BD80B5A6490968002914D079
:1043EC00C0B2002807D0A34800680179A148006832
:1043FC00083001F05FF89F480068FFF716FC0020BA
:10440C009C49086000209C49087001BD80B501885A
:10441C00012902D0022904D007E0807800F00DF8C1
:10442C0003E0807800F084F8FFE701BD80B501005F
:10443C00C9B2012000F0C2F801BD10B58AB0040069
:10444C00E4B2200001280AD0022842D004284ED021
:10445C00052856D006283DD0072847D05DE006A891
:10446C0002A94FF4417001F0FFFD9DF808008DF892
:10447C0000009DF809008DF801009DF80A008DF8E8
:10448C00020000208DF8040000208DF803009DF838
:10449C000D008DF807009DF80C008DF806009DF8B6
:1044AC000B008DF805006A460821002002F080F907
:1044BC0002A801F062FC0100704802F089FD02A91B
:1044CC0006A800F077FB0C2206A9812000F0AAFBBD
:1044DC0023E022E004A940F2153001F0C5FD0120D3
:1044EC0061490870072000F08FFC16E015E01420DD
:1044FC00FFF771FF00205C490870062000F084FC77
:10450C000BE01420FFF767FF0020574908700920C3
:10451C0000F07AFC062000F077FC4D4804700AB0DD
:10452C0010BD80B50100C9B2022000F047F801BDF2
:10453C0010B586B004006846142102F0B1FDE4B257
:10454C00002C04D16946002002F0B9FAFFE706B04E
:10455C0010BD704780B53C49098808433A4908802A
:10456C0028480068FFF73CFB01BD0000F8B50500CA
:10457C000E0014001620FFF790FB0700002F1CD034
:10458C0016210022380002F0D7F83D70E4B27D1CF1
:10459C00220031002800FEF799FE7C753A0019487C
:1045AC0001682048006801F0B5FB012805D13448AA
:1045BC000068E4B2001B32490860F1BD38B5040054
:1045CC000D000420FFF769FB002809D0E4B2048039
:1045DC00857002000B4801681048006801F09AFBD6
:1045EC0031BD0000140900202C200940183E002089
:1045FC001A3E002018090020D4190020103D00207C
:10460C00103F0020143F00202C3F0020D08D0000D4
:10461C0024090020B83E0020C43E0020183F002092
:10462C00D03E00201C3F0020D03D0020440900203B
:10463C00D0080020B8090020B4090020E43E002076
:10464C00AC3D0020F43D00202E3F0020E08D00000A
:10465C00333F0020E88D00008C01001080A903007E
:10466C00F08D0000F88D0000353F0020D88D000043
:10467C00883D0020203F0020343F0020408D00006A
:10468C00E03E002070B582B006000D001400002042
:10469C00009004226946832000F00DFB00983060E6
:1046AC000020009001226946842000F004FB009851
:1046BC00052802D1002028600DE00098062802D1C0
:1046CC000120286007E00098072802D1022028600A
:1046DC0001E003202860002000900122694685201B
:1046EC0000F0E9FA0098022802D10120206001E0D4
:1046FC000020206073BD000030B4DFF83C27127836
:10470C00642A03DB0022DFF830371A70002207E03E
:10471C00DFF824371B785B1CDFF81C472370521C16
:10472C008A4248D2835CDFF81447DFF80C572D78A7
:10473C006355DFF80837DFF8004724781B5D0D2B35
:10474C0009D1DFF8F836DFF8F0462478234413F863
:10475C00013C0A2B11D0DFF8E436DFF8DC46247874
:10476C001B5D0A2B12D1DFF8D436DFF8CC46247847
:10477C00234413F8013C0D2B08D1DFF8BC0600785C
:10478C00401CDFF8B4160870002015E0DFF8AC36DA
:10479C00DFF8A44624781B5D082BB9D1DFF89836D6
:1047AC001B78002B06D0DFF890361B785B1EDFF8E9
:1047BC0088462370B3E7012030BC704770B582B0D7
:1047CC0004000D000020009029002000FFF794FF4A
:1047DC0000287BD1DFF86446DFF85C060578DFF84B
:1047EC0060060068FEF72AFD0100C9B2200000F047
:1047FC00A2F8DFF84C060068FEF720FD0200DFF897
:10480C0040060168200002F02BFC00280BD0002091
:10481C00DFF82416087064210022DFF820462000FF
:10482C0001F08AFF52E0DFF818060068FEF706FD7B
:10483C002D1ADFF810060068FEF700FD2D1A002671
:10484C0000E0761CAE4209D2DFF8F4050068FEF7F2
:10485C00F5FC2044805D2028F3D13500DFF8E0051D
:10486C000068FEF7EBFC2900C9B2204400F063F8A5
:10487C0000261EE0DFF8C8050068FEF7DFFC2A0002
:10488C00DFF8C41551F83610204402F0E9FB00287B
:10489C000ED1DFF8AC050068FEF7D0FC20442844AC
:1048AC0000906846DFF8A01501EBC60149688847FF
:1048BC00761C062EDED30020DFF87C1508706421F0
:1048CC000022DFF87845200001F036FF73BD30B5CB
:1048DC009BB0DFF8780502F07BFB002427E0642115
:1048EC00002201AD280001F027FF6A4601212000BB
:1048FC008038C0B200F01EFF01AA9DF80000411CD8
:10490C00C9B220008038C0B200F014FF0DF10503CD
:10491C00DFF83C05210108444268DFF83405210129
:10492C00405A411CDFF82C0502F052FB641C102C81
:10493C00D5DB1BB030BD0AE0491EC9B2425C413A1E
:10494C001A2A04D2C9B2425C2032C9B24254C9B24A
:10495C000029F1D1704702E00268521C0260026823
:10496C0012780B00DBB29A42F6D0704738B50400CF
:10497C00002020212000FFF7EEFF206800780D2892
:10498C0003D0206800780A2802D1FFF7A0FF45E089
:10499C00032286A1206802F063FB002806D00322C4
:1049AC0083A1206802F05CFB002837D12068C01C72
:1049BC00206030212000FFF7CEFF206802F073FB4F
:1049CC000500A81E08281FD201202168C0B2084487
:1049DC00206020212000FFF7BEFF3D212000FFF7C3
:1049EC00BAFF20212000FFF7B6FF2068FEF726FC57
:1049FC00821E216815F17F0000F014F900280AD0FE
:104A0C00032000F001FA09E0B5F10A00062801D2F2
:104A1C000220DAE702E0042000F0F6F931BD30B5EF
:104A2C009BB0022432E06421002201AD280001F089
:104A3C0083FEDFF81C04210108448068FEF7FEFBAE
:104A4C008DF800000122694601AD2800FEF73EFCFE
:104A5C00DFF8FC03210108448068FEF7EFFBDFF868
:104A6C00F0132201114489680DF10505020028009C
:104A7C00FEF72CFC01A8FEF7E1FB01AA0100C9B26C
:104A8C0020008038C0B200F06AFE641C102C02DAE0
:104A9C00082CC8D1F9E7002000F067F81BB030BD36
:104AAC0030B59BB06421002201AC200001F044FE23
:104ABC006A460121802000F03DFE01AA9DF800000D
:104ACC00411CC9B2802000F035FE9DF800200DF18C
:104ADC000501DFF87C03806802F0C2FA002807D1D8
:104AEC009DF80000002803D09DF80000642836DBF8
:104AFC00002432E06421002201AD280001F01CFEEC
:104B0C00DFF84C03210108448068FEF797FB8DF811
:104B1C0000000122694601AD2800FEF7D7FBDFF843
:104B2C003003210108448068FEF788FB0200DFF89F
:104B3C0020032101084481680DF105052800FEF7CA
:104B4C00C5FB01A8FEF77AFB010001AAC9B220003F
:104B5C008038C0B200F003FE641C102CCADB1BB002
:104B6C0030BD80B501F029FB01BD80B5002000F0FF
:104B7C00CDFD012000F048F901BD80B5B64801F02B
:104B8C009BF8082000F040F901BD80B5B3480078CF
:104B9C00062803D0B1480078072805D10120B04978
:104BAC000870072000F030F901BD0000766172003A
:104BBC005641520070B584B004000D000C21002247
:104BCC006E46300001F0B8FD002005210CE06A5C57
:104BDC00D2B212096B461A546A5C12F00F026B4681
:104BEC0003445A70801C491E0C28F0DB002004E0A2
:104BFC006946095C30312154401C0C280FDA694697
:104C0C00095C0A29F4DB6946095C0A39062904D2D5
:104C1C006946095C37312154EEE7002000E00120A1
:104C2C0004B070BD74B599B004000D00199800283B
:104C3C0002D01998642801D3002029E02000813883
:104C4C0028D0401E05D0401E25D0401E0A282FD942
:104C5C002FE0642100226E46300001F06DFD012230
:104C6C0019A96E463000FEF731FB1998421C0DF164
:104C7C00010629003000FEF729FB6846FEF7DEFA34
:104C8C006A460100C9B22000C0B200F068FD0120E4
:104C9C001AB070BDDDE7280002F005FA4FF49661FA
:104CAC0090FBF1F201FB1200002801D00020EFE78D
:104CBC00CFE70020ECE7F0B59BB006000C00150028
:104CCC00002000906421002201AF380001F034FD77
:104CDC00002D00F09680642D80F093803000803899
:104CEC0009D0401E1CD0401E05D0401E61D0401E75
:104CFC000A2872D985E06A4601213000C0B200F062
:104D0C0019FD01AA0098411CC9B23000C0B200F0D4
:104D1C0011FD009A0DF105012000FEF7D7FA70E0A5
:104D2C006A4601213000C0B200F004FD01AA0098CF
:104D3C00411CC9B23000C0B200F0FCFC012005E0FF
:104D4C0001A9095C303901AA1154401C0099491C75
:104D5C0088421CDA01A9095C30390A29F0D301A96F
:104D6C00095C4139062905D201A9095C373901AA28
:104D7C001154EAE701A9095C6139062905D201A998
:104D8C00095C573901AA1154DFE700203AE00020F2
:104D9C0000990AE001AA0A4412F8012C01AB5B5CF1
:104DAC0053EA02122254401C891EA842F2D301205D
:104DBC0028E06A4601213000C0B200F0BBFC01AA19
:104DCC000098411CC9B23000C0B200F0B3FC0DF128
:104DDC00050002F068F9206013E06A4601213000FA
:104DEC00C0B200F0A7FC01AA0098411CC9B2300067
:104DFC00C0B200F09FFC0DF1050002F054F92080C8
:104E0C00FFE700201BB0F0BD10B582B004000020FD
:104E1C008DF80000012269468720FFF74CFF9DF8B2
:104E2C000000002806D00F48E4B250F824100E48B9
:104E3C0002F0CEF813BD0000323F0020AC3C002045
:104E4C00AC090020B00900204CF701001CF7010050
:104E5C0060F10100448C0000F43D0020333F002041
:104E6C00353F0020080800209C8D0000E0B508218B
:104E7C00ADF800100190022100F00FF8002814BFCB
:104E8C00002002980EBD00B583B00821ADF80010CB
:104E9C000190032100F001F807BDADF8021068463F
:104EAC00DFF87813096808471FB5ADF80610ADF8A0
:104EBC0004000824DFF864138DF808200393ADF880
:104ECC000040ADF8024068460968884704B010BD40
:104EDC0030B585B0144608220291ADF80020192295
:104EEC00DFF8381309680190ADF802201D466846BA
:104EFC00884714B1BDF80C10218015B1BDF80E1007
:104F0C002980089A0499116005B030BD00B583B0B2
:104F1C000820ADF800001A2000F014F800280CBF8F
:104F2C00BDF80400FF200EBDE0B5ADF80000ADF8F3
:104F3C000610002000F006F800280CBF9DF80800B1
:104F4C00FF200EBDDFF8D4120968ADF802006846E8
:104F5C00084750B110F1040F01D10420704710F133
:104F6C00030F01D102207047012070478123037089
:104F7C0042EAC111002341F47C41C3708180704727
:104F8C008223037081800023C370827170473EB509
:104F9C0004460820ADF800000D462020ADF80200B4
:104FAC001020DFF878120968ADF8040068468847CD
:104FBC0020B9029810B16FF004003EBD009500239B
:104FCC00002221464FF0FF30FFF782FF3EBD10B5A7
:104FDC0082B01446CA78012A03D18A88DFF8E834F3
:104FEC001A8000F010F858B9009069462046FFF777
:104FFC00CEFF28B900984478FFF745FF204616BD30
:10500C00FFF7A7FF16BD0B46022210214CE738B55F
:10501C001C461546FFF7F7FFC0B9009069462846B5
:10502C00FFF7B5FF90B900984578280002BF0098AB
:10503C00C079A04205D10098816804982246FEF7F9
:10504C0045F90098FFF71FFF284632BDFFF781FF97
:10505C0032BDF8B500F057FA00F0C0F907000DD0DA
:10506C0032462946FFF78CFF00F049F93872FFF7FA
:10507C004DFF3B4601B0BDE8F0403AE0F1BD1022D7
:10508C000121E6E738B500F0E2F9050004D004226E
:10509C0000F032F8AC6026E031BD3C81BD72FE60A0
:1050AC0034E72DE9F04100F05BF907000FD0142232
:1050BC0000F022F83C72FD603E8287F81280FFF708
:1050CC0025FF3946BDE8F041DFF800247FE72FE0EB
:1050DC0038B500F033F8050001D0152200E031BDE1
:1050EC0000F00AF82C81FFF711FF2B4601B0BDE848
:1050FC00304002221021D7E6012141E70022042191
:10510C0077E02DE9F04100F02BF9070010D00222D6
:10511C000421FFF735FFBC60BD81BE73C7F810805A
:10512C00FFF7F4FE3946BDE8F041DFF8A4234EE763
:10513C000420BDE8F081102202218AE704460A20EF
:10514C0094E602211CE7F8B500F07BF907000AD0C1
:10515C001522FFF7F6FFFFF7A0FF3946BDE8F84030
:10516C00DFF8702333E70420F2BD0022032140E076
:10517C0000B583B00FF24903019306230093032378
:10518C0000F04EF80EBD1078802802BF508840F217
:10519C007F61884208D19088984202BF917900982B
:1051AC00814201D1012070470020704710B582B0B8
:1051BC000624FFE70094FFF7E6FF16BD0000000091
:1051CC000323F3E71078802802BF508840F27F61F8
:1051DC0088420CD19088032818BF042807D19079F5
:1051EC0001001CBF1028112801D10120704700209C
:1051FC007047F8B500F013FA07000CD03246294678
:10520C00FFF7BEFEBC60FFF781FE3946BDE8F840F3
:10521C00DFF8C422DBE60420F2BD000014090020F4
:10522C002DE9F04100F027F807000AD0069A414614
:10523C00FFF7A6FE3C817D81FFF731FF079A00F056
:10524C0027BA75E74246032190E670B582B000F0AC
:10525C005AF9FFF75BFE1B210091C3B23246294677
:10526C00204600F0FEF876BD10B582B01D240094E7
:10527C0000F0F7F816BD04460D4616469846102069
:10528C00FFF7F4BD2DE9F04180460D4616461F464A
:10529C001820FFF7EBFD040014D0002200F05DF89D
:1052AC0000F030FA20726572A672E76006982061F1
:1052BC0007986061FFF72AFE2146BDE8F0410FF226
:1052CC00BD2284E634E70FF2B923112200211EE13E
:1052DC00F8B500F0C0F807000FD00A2200F03DF836
:1052EC0000F00DF838727D813E73FFF70FFE3946E2
:1052FC00BDE8F8400FF28D2269E60420F2BD21468C
:10530C005020FFF711BE0FF28123062210E12DE988
:10531C00F04180460D4616461F461020FFF7A6FDAD
:10532C00040010D0072200F018F800F0EBF92072FE
:10533C006572A672E760FFF7E9FD2146BDE8F04112
:10534C000FF2492243E6F3E60FF24523082200212F
:10535C00EEE00FF241231022C4E00421FFF706BE59
:10536C0004460D46164698461420FFF77FBD70B5CF
:10537C0000F014F806000BD03022FFF7EEFF00F01F
:10538C0009F83146BDE870400FF20D22FFF71FBE41
:10539C00042070BD34817581FFF7B8BD04460D46FD
:1053AC000C20FFF763BD30B583B004460020ADF888
:1053BC00040000F013F805000DD03122FFF7CDFFEB
:1053CC002C81FFF7A3FD01A9009102230FF2CD124E
:1053DC002946FFF71CFEBDF804003EBD0A20FFF76E
:1053EC0045BD1CB500208DF8040000F012F8040037
:1053FC000CD01222FFF780FEFFF788FD01A9009167
:10540C0001230FF29D122146FFF701FE9DF80400C7
:10541C0016BD0820FFF72ABDF8B500F012F80700FA
:10542C000DD03622FFF799FF3C817D81FFF737FEC7
:10543C003946BDE8F8400FF27912FFF7C8BD0420D9
:10544C00F2BD04460D4616461020FFF70FBD04466C
:10545C000C20FFF70BBD04460D4616460E20FFF739
:10546C0005BD2DE9F041FFF77BFF070011D0069A2F
:10547C00FFF7E9FE3C813E74FD6000F043F978745F
:10548C00FFF744FD3946BDE8F0410FF25912FFF722
:10549C009EBDFFF74DBE38B51446104A15682A005C
:1054AC0006D0009302460B4621460120A84732BD88
:1054BC00002032BD0A4A13681A0003D00A4601467E
:1054CC000120184770470000C40900201156000045
:1054DC002156000017560000D1510000FC3E002060
:1054EC00003F00202DE9F04100F00DF898460C200B
:1054FC00FFF7BCFC070004D000F016F83C81BD722D
:10550C00C3E0FFF715BE04460D46164670472DE95D
:10551C00F041FFF7B0FE070004D000F005F8BC60C6
:10552C00FD60B2E0FFF704BE32460421FFF71EBD5A
:10553C002DE9F041FFF79FFE070006D0FFF7F4FFBF
:10554C00FFF7DDFE3872FD609FE0FFF7F1BD1078CC
:10555C00802802BF508840F27F6188420CD190882D
:10556C004FF680710140B1F57E4F04BF00F07F0013
:10557C00984201D101207047002070470023E6E7D4
:10558C001123E4E70A23E2E70623E0E70723DEE73B
:10559C000823DCE71023DAE73023D8E73123D6E7FA
:1055AC0080B5122300930123FFF7EDFD02BD00002F
:1055BC003623CCE71078802802BF508840F27F61F8
:1055CC0088420DD190884FF6807101404FF6805281
:1055DC00914204BF00F07F00984201D10120704736
:1055EC000020704770B5FFF78EFF1D23FFF7E2FF19
:1055FC0030B9324629462046BDE870401B23D9E716
:10560C00012070BD80B51423CCE780B51523009321
:10561C000223C9E780B5022300930423C4E70446A0
:10562C000D4616460C20FFF721BC2DE9F041FFF783
:10563C006AFF98460E20FFF719FC070009D000F00E
:10564C001CF83D817E81A7F80C80FFF75FFC069A61
:10565C001EE0FFF76DBD2DE9F041FFF781FE07005D
:10566C0009D000F00AF8BD60FE60C7F81080FFF7A3
:10567C004DFC069A0CE0FFF75BBD812038700120D1
:10568C00F870BC8070473D81FE60FFF73FFC4246DE
:10569C003946BDE8F041FFF79ABC1078802802BF6C
:1056AC00508840F27F61884204BF9088984201D1B3
:1056BC000120704700207047FFF7B7FF02BD009133
:1056CC000023014600227047FFF7C5FF02BD80B5DD
:1056DC000FF24901FFF7F3FF4FF60C40F4E738B532
:1056EC000446154600F00FF80FF239010091C2B2D2
:1056FC002B4621464FF61840FFF797FF32BD3C81F1
:10570C007D81BE8141465020FFF70EBC80B50FF263
:10571C001D01FFF7D4FF4FF61D40CDE74FF60C43AC
:10572C00BBE700004FF61843B7E700004FF61D43E8
:10573C00B3E70000F8B5FFF784FE07000DD0012297
:10574C0000F022F83C727D72FFF7A9FC3946BDE8E7
:10575C00F8400FF26D02FFF73ABC0420F2BDF8B529
:10576C00FFF76FFE07000DD0022200F00DF83C721F
:10577C007D72FFF794FC3946BDE8F8400FF2450204
:10578C00FFF725BC0420F2BD0521FFF7EFBB107815
:10579C00802802BF508840F27F6188420DD19088EA
:1057AC004FF6807101404FF68062914204BF00F0C9
:1057BC007F00984201D10120704700207047000003
:1057CC000123E4E70223E2E7DFF800F0CDA00110AB
:1057DC00DFF800F0C1C10110DFF800F03DC101108D
:1057EC00DFF800F029AF0110DFF800F009B7011065
:1057FC0090FAA0F0B0FA80F0704780B5DFF8F803AB
:10580C000068FFF7F5FF0121DFF8F02381401160FC
:10581C000121DFF8EC231160DFF8E8130A689042ED
:10582C000BD201EB80014A683AB11368190004D01D
:10583C00C1B21046BDE80440184701BDF8B50D00D3
:10584C00ECB244BF85F0204585F4C045A10001F1C0
:10585C00804101F5012100EA05060A68DFF8A8730A
:10586C003E4085EA020382433243034000F4E026C3
:10587C001B0EB6F5E02F03F0010302D1D30105D4C2
:10588C0011E010F4E02F08BF002B0CD002F4E02341
:10589C00B3F5A02F04D0B3F5C02F04D1052300E03D
:1058AC00062363F312420A60410205D5A90DDFF805
:1058BC005C2301F00101115500020ED5FCF726FA0C
:1058CC0000F057F92C024CBF1C4600249A4322438B
:1058DC000A60BDE8F240FCF71DBAF1BD002948BFD3
:1058EC000021800000F1804000F5012001F03F0113
:1058FC000268920941EA8211016070472DE9F04F6C
:10590C0097B08146FCF724FD0025012804D1FCF753
:10591C0015FD022808BF0125DFF8F402C168C1F3A8
:10592C00815101294FF0010A04D10068000E0AFAD6
:10593C0000F00543DFF8DC02DFF8C8620078DFF81E
:10594C00D8020068C0F346003060FCF701FD012866
:10595C0002D13068401C30603168DFF8C07219B178
:10596C00FF22384601F0A4FB4FF00008002405E0AC
:10597C00CC550AFA00F040EA0808641C59F82400D7
:10598C00C1B2FF2908D03268914203D225FA00F245
:10599C00D207EDD5022058E00920FBF701F9C6F833
:1059AC0080900823242200210DA8FFF711FF8DF809
:1059BC004CA00DAA012106F1A000FFF715FF002451
:1059CC00DFF85CA20BE05046FFF738FF4FF0FF31D9
:1059DC00E0B2FFF783FF0020CBF80400641C3068B2
:1059EC00844212D225FA04F0C00706EB840B48BFA0
:1059FC000420F1D428FA04F0C00747BFE05D59F841
:105A0C002010E0B240F4C041DDE708233022002131
:105A1C0001A8FFF7E1FE0020009001ABDFF80422A3
:105A2C00102106F18400FFF7DBFEDFF8FC010168B2
:105A3C0021F47C5141F4005101600120DFF8EC119C
:105A4C000860DFF8EC110860002017B0BDE8F08F9B
:105A5C002DE9F041DFF8AC6104460D4606F1A008D3
:105A6C0000F032F800273DB9002020606060A06093
:105A7C0000271DB31EE07F1C15F82700FF28F3D06C
:105A8C003168884204D206EB800040680028F2D0CE
:105A9C00002413E006EB800101224C6002FA00F0B6
:105AAC00616808436060204655F827205C4900F087
:105ABC0078F87F1C15F82700FF28EBD14046FEF73D
:105ACC008FF82046BDE8F0814FF0FF314046FFF7DC
:105ADC007BBE10B50C46F0B1416821FA04F2D20736
:105AEC0019D50122A240914341600020454901EBA8
:105AFC00840250604948225C4948FF2A0EBF44F09A
:105B0C002041D1F8801051F82210FFF797FE4FF08A
:105B1C00FF31204668E0022010BD10B5044605E0B8
:105B2C00FFF766FEC1B22046FFF7D3FF606800287E
:105B3C00F6D110BD3F49096821FA00F202F00100CC
:105B4C00704738B50C462F4915460A68944204D262
:105B5C0001EB84014968814201D0022032BDFCF77F
:105B6C00D5F800F006F89A4305FA04F31A430A60D4
:105B7C003EE031490A680123A340704710B5214B20
:105B8C001C68A14204D203EB81035B68834201D001
:105B9C00022010BD10001D4A18BF012050540020D7
:105BAC0010BD38B5174C25680B461146CAB2AA422F
:105BBC0004D204EB82025268824201D0022032BD30
:105BCC001846FFF73BFE002032BD0B4610B51146C0
:105BDC000C4A1468A34204D202EB8302526882423C
:105BEC0001D0022010BD1846FFF778FE002010BD32
:105BFC00FCF790F8002032BDE0200240E02002606B
:105C0C0080E200E0F03B0020007F077F0020024094
:105C1C00A83F0050373F002080120840383E00203B
:105C2C00007FC76707580000003009400C4009404E
:105C3C0008000940C0200240D0200240DFF800F0EC
:105C4C0085C10110DFF800F0A9C10110DFF800F0E8
:105C5C0079B5011000B583B00821ADF800100190A2
:105C6C000521ADF80210684655490968884707BDFB
:105C7C00F0B589B004460D4616461F46082324226B
:105C8C0000216846FFF7DAFF0F984E490968069025
:105C9C006B464FF47A70B0FBF1F101FB07F0059005
:105CAC0001FB06F20E98ADF8100029462046FFF7CE
:105CBC00CDFF204609B0F0BDFAF7A6BC38B50446B6
:105CCC000D46FAF756FD10B12046FAF795FC00F098
:105CDC0013F800FB05F12046FAF792FC2046BDE8CC
:105CEC003240FAF791BC80B5FAF743FD00B10120C0
:105CFC00C0B202BDFAF780BC324909684FF47A7021
:105D0C00B0FBF1F0704710B504460021FAF78CFC9B
:105D1C00204610BD70B584B004460820ADF80000D4
:105D2C000D460420ADF802000C20254909680190AD
:105D3C0016466846884758B9029949B18E60204684
:105D4C00FAF76AFC15B12846FDF74AFF012003E07B
:105D5C003046FFF77FFF002004B070BD10B504463D
:105D6C00FAF756FC38B92046FFF76CFF8468FFF74A
:105D7C0071FF204610BD002010BD30B585B0044623
:105D8C0068460FF248011422FDF7B0FA0E48302194
:105D9C000170A21D782141700623811C12F8015D4F
:105DAC002D095B1E1DF8055001F8015B157805F0F7
:105DBC000F051DF8055001F8015BEFD105B030BDA2
:105DCC0014090020208E0000803E00203031323338
:105DDC0034353637383941424344454600000000DB
:105DEC002DE9F04EDFF840799246002640F2013B57
:105DFC000C467A783B7997F803C0B7F81090B0EB63
:105E0C000B0540F67B4132D06D1E38D06D1E3DD057
:105E1C00AD1E41D06D1E00F07B806D1E00F07E80AB
:105E2C006D1E00F08A806D1E00F09A806D1E00F0D1
:105E3C009F806D1E00F0A4806D1E00F0AB806D1E67
:105E4C0000F0B080ED1E00F0B5806D1E00F0BA8041
:105E5C006D1E00F0BF806D1E00F0C4806D1E00F042
:105E6C00C9806D1F00F0D180AD1E2DD0E5E0102C47
:105E7C0040F0E1801022514607F1A40087E0102C7D
:105E8C006FD11022514607F1B40080E0042C68D188
:105E9C00DAF80000F862DBE0012C62D1012B35D07E
:105EAC009AF80000F870BCF1000F06D00028F2D16F
:105EBC00022A19D0052AEED116E00028EBD0012ACF
:105ECC0020D0042A1CD11DE0012C4AD1BCF1010FB9
:105EDC001CD09AF8000038715BB1002808D1032A55
:105EEC001CBF072A052A03D15FFA89F0FFF72CFAA9
:105EFC00AEE00028FCD0012A1CBF042A062A01D0DF
:105F0C00052A02D1012000F008FCA1E012269FE036
:105F1C00022C26D1BAF80000B88299E0202C0DDAB8
:105F2C0007F1CC061F21304601F0E0F800F093F8A1
:105F3C007C713346224601210DE0202C7BDA07F1DF
:105F4C00EC061F21304601F0D1F800F084F8BC714A
:105F5C003346224600215FFA89F0FFF7D8F974E046
:105F6C00012C68D19AF80000052864DAF8716FE00A
:105F7C00012C60D19AF8000004285CDA387267E0D2
:105F8C00062C58D14FF48670062251463844FDF742
:105F9C009DF95DE0012C4ED19AF8000008284ADAF0
:105FAC00787255E0012C46D19AF80000042842DAA8
:105FBC00B8724DE0012C3ED19AF8000002283ADA72
:105FCC00F87245E000F04CF835D1821F8A4232D28B
:105FDC0038833DE000F044F82DD1821F8A422AD24A
:105FEC00788335E000F03CF825D1B0F5FA7F22DA61
:105FFC00B8832DE000F034F81DD1A0F10A0140F671
:10600C007742914217D2F88322E0012C04BF9AF810
:10601C00000001280FD107F18000FFF764FE40B9A2
:10602C0000F020FB060013D107F15C00FFF762FEC5
:10603C000EE016260CE018260AE0272807DA022CB8
:10604C0005D1BAF80010FFF792F9064600E00226D7
:10605C003046BDE8F08E224651463046FDF736B943
:10606C00BAF80000022C704738B500244FF4407386
:10607C000D46C21ADFF8B01636D0521E36D0521E5C
:10608C0037D0521E38D0521E39D0521E3AD0521E22
:10609C003CD0521E3CD0521E3DD0521E3ED0521E01
:1060AC003ED0521E3ED0521E40D0521E40D0521EE8
:1060BC0040D0921E40D0521E40D0521E40D0521E94
:1060CC0040D0521E40D0521E40D0521E46D0521EBE
:1060DC0046D0521E46D0921E48D0521E14D0521E8C
:1060EC0042D0521E44D046E0887842E01022A431BF
:1060FC0030E01022B4312DE0C86A286042E006225C
:10610C00C43127E0C87834E0087932E0888A36E078
:10611C004A79CC311EE08A79EC311BE0C87928E051
:10612C00087A26E006224FF4867012E0487A20E0C6
:10613C00887A1EE0C88A22E0C87A20E0088B1EE02C
:10614C00488B1CE0888B1AE0C88B18E006224FF4B1
:10615C008A7001442846FDF7B9F813E0088C0EE06C
:10616C00488C0CE0888C0AE0087B02E0487800E060
:10617C00487B287006E0272803DAFFF714F92880FB
:10618C0000E00224204632BD1CB5DFF89C45617846
:10619C0089B900B1206304F12C00019004F1B40022
:1061AC00009004F1A403208AA1780022C0B2FFF76A
:1061BC0069F8002016BD112016BDDFF86C0541787A
:1061CC00062918BF072905D1C18A008A1322C0B23B
:1061DC00FFF77EB81220704700B58FB008233C2221
:1061EC0000216846FDF7F8FCDFF8400500F150018E
:1061FC000791002340F2EE2108916A460321069193
:10620C000FF2CD01FDF7F0FC0FB000BD70B584B0FE
:10621C0000F016F90120DFF81815DFF80C450968B5
:10622C000FF21155ADF80200002668468847BDF8FC
:10623C00040020820298A062002060704FF6FF706C
:10624C00E082FFF7CEF8207000230120019000229D
:10625C0000200090294604F13800FFF709FD0220C8
:10626C0000F02FF804F15C00FFF702FD042000F0B1
:10627C0028F804F18000FFF7FBFC0420A07004F167
:10628C00A40200200021002300252BC204F1B40538
:10629C00103A4BC5E062E0712072A1720720607267
:1062AC0010210220FFF746FA103D2A461021032048
:1062BC00FFF740FA04F12C0204210420FFF73AFA0C
:1062CC007FBD0190002300200090002229467047DA
:1062DC00FEB5FFF79BFFDFF85054DFF8544405F18F
:1062EC00800700F0ADF80A20ADF802004FF0FF3047
:1062FC00019068462168884700284BD100F0A0F82F
:10630C000920ADF80200684621688847BDF80610E0
:10631C00029E00283ED1BDF80400102804BF288A34
:10632C0081422DD130884FF6FF71884209D1708897
:10633C00400425D505F12C0204210420FFF70FFAA7
:10634C001EE03078A22805D0D02804BF304600F0DB
:10635C007BF815E07079132812D13089012804BF1D
:10636C00A87B022805D13846FFF7C4FCFFF725FFB0
:10637C0006E00520FFF717F801463846FFF79EFCAC
:10638C0046B100F05DF80320ADF8020001966846B6
:10639C0021688847688AC10731D54FF6FE710840DD
:1063AC006882E9782879014329D018B103208DF847
:1063BC0000000DE0E8798DF800000622287A8DF8AF
:1063CC0001004FF4867029180DF10200FCF77EFFD6
:1063DC00687A8DF808006946A87A8DF80900288A31
:1063EC00C0B2FEF790FF00281FBF08206870286B12
:1063FC00002804D0016808001CBF08208847688A60
:10640C00810706D54FF6FD7108406882002000F028
:10641C0029F9688A41070AD54FF6FB710840688252
:10642C00A87B012804D0022808BFFFF7C6FE58E756
:10643C000090EB8BAA8B698B288B00F047F950E707
:10644C000820ADF800007047F8B50546B64CA878A2
:10645C004FF48A716718010004F1800612D00228EB
:10646C003CD0032818BF04285CD0052800F082809B
:10647C00062800F0AD80072800F0CF800F2800F030
:10648C00EB80F1BD687801001BD104F1A40210214E
:10649C000220FFF764F904F1B40210210320FFF786
:1064AC005EF90622E91C04F1C400FCF70FFF012081
:1064BC00607004F1CC03208A62790121C0B2FEF72E
:1064CC0026FF08B108206070206B30B1016808000D
:1064DC0003D06078BDE8F4400847F1BD6878E8B9AE
:1064EC00E87848B1208AA27904F1EC030021C0B20B
:1064FC00FEF70DFF687011E06078022818BF0728BE
:10650C000CD0062802D12079012807D104F13800DB
:10651C00FFF7E9FB10B9012000F0FFF868780028BC
:10652C00DBD0CFE7697821BB03280AD16078062835
:10653C0008BF0720C7D0E07800280CBF032002203A
:10654C00C1E7A18A0800E07807D0227910430AD06D
:10655C0004F13800FFF7B2FB05E0012807BF00206B
:10656C00E070002020716078072814BF04200620FA
:10657C00A9E7A7E76878010024D10622291D38462F
:10658C00FCF7A4FE6889E08206206070E88920840C
:10659C00288A6084688AA084E8782073E07A0128CD
:1065AC0009D11F20FEF7FFFE4FF47A71414304F12D
:1065BC005C00FFF783FB6A89E8780423291DFEF74A
:1065CC0070FD81E73128D4D10020E07004207AE7F7
:1065DC00A888FEF77DFD0621384600F087FD0020D7
:1065EC0020846084A084A879607304F15C00FFF7B8
:1065FC0081FB3046FFF77EFB4FF6FF70E08220797F
:10660C0008B103205FE7A87908280CBF05200420F7
:10661C006070012000F081F856E73046FFF76AFB06
:10662C00687800280AD1E8882084288960846889E1
:10663C00A08404F15C00FFF756FB00287FF44DAFFB
:10664C00636B002B3FF449AF1B68A28C618C208CD0
:10665C0001B0BDE8F0401847A888BDE8F44005211A
:10666C00FEF777BEFEB5304D2A8B0446288C90423F
:10667C0024BF698B814207D3688CA98B884202BFE7
:10668C00A88CE98B88421ED00520FEF78CFE0646AE
:10669C00E88AADF80000288BADF80200688BADF8E5
:1066AC000400A88BADF80600E88BADF8080068462E
:1066BC00FEF709FE070007D1AC73314605F18000E7
:1066CC00FFF7FCFA00E018273846FEBD70B5164CF3
:1066DC006578062D01D0142070BD40F67A45861FD2
:1066EC00AE423CBF8E1FAE4215D2B2F5FA7F12DA23
:1066FC00A3F10A0540F67646B5420CD2208361839D
:10670C00A283E3830498FFF7ADFF04F15C00FFF76D
:10671C00F1FA002070BD182070BD03494A8A10435D
:10672C004882886AFDF75CBA38030020A02E00204E
:10673C0014090020F1E7000062F30F2262F31F42FC
:10674C00401810F0030308D0C91A1FD3DB0748BF49
:10675C0000F8012D28BF20F8022D130030B4144688
:10676C001546103928BF20E93C00FAD8490728BF44
:10677C0020E90C0048BF40F8042D890028BF20F800
:10678C00022D48BF00F8012D30BC7047C91818BF46
:10679C0000F8012DCB0728BF00F8012D7047000031
:1067AC000FF204237D4810221321FEF7AABC00002F
:1067BC002DE9F0430024082885B00E469146784F09
:1067CC0000F28A80DFE800F0050C1824303C4853B6
:1067DC007D00082E76D13246494607F1080076E056
:1067EC00152E77DA152107F1100000F059FC32460E
:1067FC00494607F110006AE0152E6BDA152107F1F6
:10680C00280000F04DFC3246494607F128005EE0B6
:10681C00152E5FDA152107F1400000F041FC3246DD
:10682C00494607F1400052E0152E53DA152107F1C5
:10683C00580000F035FC3246494607F1580046E056
:10684C00152E47DA152107F1700000F029FC3246AD
:10685C00494607F170003AE0152E3BDA88371521CE
:10686C00384600F01DFC3246494638462FE00820D9
:10687C00ADF808000420ADF80A00039602A8DFF872
:10688C002481D8F800108847C8B9049DBDB1786838
:10689C0007F1A00188420AD00821ADF80010019040
:1068AC000521ADF802106846D8F80010884732462A
:1068BC0049462846FCF70AFD7D603E700DE0132426
:1068CC000BE0072E06D13246494607F1B000FCF723
:1068DC00FDFC02E0182400E00224204605B0BDE8CF
:1068EC00F08300002DE9FE4990464A680A9C107816
:1068FC0052780B9D00EB02201F46002680B242F618
:10690C002322274B801A03EB040C07D0401E0528CA
:10691C0010D9801F1ED0263829D03AE0092C28D255
:10692C00C4F10800854228BFC4F108053D800CF174
:10693C00080129E0D1F80CB05846FCF77FFC80B276
:10694C00A04216DB011B8D42A8BF051B3D800BEB43
:10695C00040119E018780146A1420AD3001B8542B4
:10696C00A8BF0D1B3D8058683A8801190DE0082C12
:10697C0001D307260FE0C4F10700854228BFC4F1FC
:10698C0007053D800CF1B0013A884046FCF79EFCAF
:10699C0001E03E800A263046BDE8FE890802002050
:1069AC005404002014090020F168000000000000CD
:1069BC00000000003EB504460820ADF8000004209D
:1069CC00ADF802008349844800780968834D800043
:1069DC00019068468847002814BF002002980100E7
:1069EC00686001D113203EBD4FF6FF7000F082FBB2
:1069FC00E00708D50FF2FC131022092105F11C0049
:106A0C00FEF77FFB3EBD00203EBD00281DBF744934
:106A1C00086000201120704770B584B00C461546F4
:106A2C0000BB152C1CDA6D4E142106F1080000F089
:106A3C0037FB2246294606F10800FCF747FC0FF20B
:106A4C00990002903470FF20019006F11C0309207C
:106A5C0000900022706806F1080100F065FB02E06E
:106A6C00182000E0022004B070BD0021020004D008
:106A7C005C4A1368C018106000E018210846704783
:106A8C00012859490BD0022805D0082802BF0868F4
:106A9C00401C086006E08868401C886002E048687A
:106AAC00401C4860002070470021020004D04F4A6F
:106ABC001368C018106000E018210846704710B524
:106ACC000B46002428B9142249491846FCF7FEFB52
:106ADC0000E00224204610BD38B510460A7A002486
:106AEC00D20601D5082032BD049A0AB10B2032BD62
:106AFC000A78102A12D14A68157B527B05EB0222C8
:106B0C0092B24CF2E105AA4206D1344A12781A80AC
:106B1C00C968FCF7DBFB07E01C8002E0022A1C8042
:106B2C0001D10A2400E00124204632BDF0B583B027
:106B3C0015460A7A002492061E4601D50820FEBD91
:106B4C000B78089A102B2CD14B68187B5B7B00EBD5
:106B5C00032080B24CF2E103984230D11AB9152EC1
:106B6C0003DB0D241BE00B2419E0CF6814213846FD
:106B7C0000F0BCFA324629463846FCF7A7FB3146F2
:106B8C00384600F0EDF9300018BFFFF78DFF1448C0
:106B9C00006820B1016808001CBF0020884720460F
:106BAC00FEBD022B18BF0124F9D14B681C785B7811
:106BBC0004EB03239BB242F60214A34201D00A2435
:106BCC00EDE701230193009233462A4600F00FFBB8
:106BDC000446E4E714090020380300200C050020CB
:106BEC00043F0020083F0020AC3E00200C3F00205A
:106BFC0014050020E56A0000396B0000000000005D
:106C0C0072494862704738B57148704D00688047CA
:106C1C000446686900F098FB686900F07DFB20462B
:106C2C00BDE834406B490968084738B5FFF7EBFFFE
:106C3C0000F05BF804466849002000F073FB6349E0
:106C4C0048610022202100F06AFB00F092F8054612
:106C5C002046884700F090F8E8B232BD38B55B4C5E
:106C6C005D4DE0612162A261284600F065FB4FF4A6
:106C7C00E130A861294600206875A87503202877A3
:106C8C00002068770120287068700020E8750FF2EA
:106C9C006100E8600FF219002861002000F042FB4F
:106CAC0060610022BDE83840202100F038BB0000B4
:106CBC0038B5054600F019F804466868434DC07FA6
:106CCC008DF8000030B16B6A180003D001226946C0
:106CDC0020209847AA69100002D0698A00209047AA
:106CEC0000F047F82046884731BD39480068004716
:106CFC00F8B5064636480068144680470546706865
:106D0C00324EC07F8DF8000030B1736A180003D08A
:106D1C000122694620209847CCB1318A002089B2E3
:106D2C00B1F5007F09DAF769335C7B5400223254E9
:106D3C00401C491CC0B2A042F1D38442318206D01F
:106D4C00B269100009D0718A4FF400709047B26993
:106D5C00100002D00021A0B29047002030821022F7
:106D6C007069314600F0EDFA00F003F828468847C8
:106D7C00F1BD18490968704710B5FFF7B6FF044616
:106D8C001249002008821022486900F0DAFA2046E5
:106D9C00FFF7EFFFBDE81040084770B504460C48FC
:106DAC000A4E006880470546316A70697482224633
:106DBC0000F0CDFA074910F1010F04BF00207082DA
:106DCC00096828468847708A70BD0000603D002025
:106DDC000C09002010090020AC3D0020DFF800F069
:106DEC0021B90110E0B500F010F8042100F012F800
:106DFC00002814BF002002980EBD00B583B000F02F
:106E0C0004F8052100F006F807BD0821ADF80010C4
:106E1C0001907047ADF8021068468D490968084723
:106E2C0030B58C4C0020A06087B00021FFF7D6FF56
:106E3C0060600823182200216846FBF7A8F84FF47D
:106E4C000570251869462846FBF7A5F8E5600FF292
:106E5C00F5120FF2D9110FF2B51000F08DFA07B040
:106E6C0030BD70B57B4C22E020704FF4007104F102
:106E7C00140000F015F9217804F1140000F060FB07
:106E8C002369180004D0227804F1140110209847CB
:106E9C006088152803DBE0680121F9F709FDA807D4
:106EAC0005D56068F9F7B4FB08B900F08DF8E06817
:106EBC004FF0FF330F220021F9F78AFC05466807D3
:106ECC001DD56068F9F7A4FB98B900F06FFA80B98A
:106EDC006068FEF7B7FE06000BD0B1684868A0608A
:106EEC00497800F09DFAB068FFF787FF3046FFF74E
:106EFC0084FF6068F9F78CFB08B900F065F8E807C7
:106F0C00CDD500F00FFB15286080ADDB1420ABE76E
:106F1C0080B5FFF785FFBDE80140A2E730B54E4CC8
:106F2C004FF400758FB0DD22294604F1500000F0BB
:106F3C00BFF808233C2200216846FCF74DFE04F103
:106F4C005000079008950220069000236A4643499A
:106F5C002046FCF749FE0FB030BD3E490861704732
:106F6C00FEB504460D46FF20FEF7E4FD58BB082095
:106F7C00FFF738FF06001DD0002030700820ADF858
:106F8C000000022032490968ADF8020001956846FC
:106F9C008847002814BF00200298706075707068D4
:106FAC0018B12A462146FCF791F90C20FFF71AFF7D
:106FBC000746BE60307830B9264C60683946F9F720
:106FCC002BFB00F001F8F7BDE0680421F9F770BC69
:106FDC000EB410B5ADF5806D81B004464FF48061F0
:106FEC00684600F05DF8FFAA10322146684600F0B2
:106FFC00C7FA6846FCF722F981B26846FFF7B0FF82
:10700C000DF5806D01B010BC5DF810FB1CB5114C7A
:10701C00A06830B1FFF7F9FE0321FFF7FBFE00205B
:10702C00A0600221E068F9F743FC13BD80B580B283
:10703C0000F040FA0748C068BDE804400121F9F7A8
:10704C0037BC00000348C0680821F9F731BC0000C8
:10705C001409002030340020E03100201D6F0000A6
:10706C0010B401E0491C521E6AB10B7804789C42A2
:10707C0005D010BC2CBF01204FF0FF30704710F82A
:10708C00013B002BEED110BC002070470246034898
:10709C000068FF21FEF772BD0000000050080020C0
:1070AC00002200F009B80A22002100F023BB0000E6
:1070BC0062F30F2262F31F4200B500BF1300964625
:1070CC009446103928BFA0E80C50FAD85FEA417CEE
:1070DC0028BF0CC048BF40F8042BC90728BF20F8B4
:1070EC00022B48BF00F8012B00BD00000022FFF767
:1070FC0027BB000038B54FF6FF74A0420DD100201D
:10710C00654A137898420EDA21F8204001EB80058D
:10711C000023401CAB70C0B2F3E700F0A9F810B12B
:10712C0004800021817031BD2DE9FE4F8046002680
:10713C00B8F1000F82B006D0080004D0180002D0BD
:10714C00109F380001D1022035E00F9C00252CE067
:10715C00EDB2A94638F829004FF6FF7188421EBFE0
:10716C0008EB890A9AF8020000281DD0029ABDF893
:10717C003810049800F02AF85FEA000B14D09AF843
:10718C000200C00705D500F019F8012100F086F8BF
:10719C0006439AF80200800706D500F00FF802218A
:1071AC0000F07CF80643F6B26D1C3B490978E8B256
:1071BC008842CDD3F0B205B0BDE8F08F01970094B2
:1071CC009DF80C2038F829005B46704730B5002438
:1071DC0000E0641CA3B28B4207D2A4B200EB0413F0
:1071EC00DD689542F5D1184630BD002030BDF8B5AC
:1071FC00044606980D460026F0B9022B1AD11078D9
:10720C00517800EB01270798C043B9B201420FD166
:10721C00E8680168204600F012F8B9B288420CD038
:10722C00E8680168BAB2204600F00FF8064604E0A0
:10723C00802602E00D2600E00B263046F2BD80B51C
:10724C0000F016F800B1807802BD70B504460D460A
:10725C00164600F00DF840B929464FF6FF7000F0C5
:10726C0007F808B9112070BD04808670002070BD2D
:10727C0010B5002200E0521C074C2478D3B2A34274
:10728C0007D2D2B231F822308342F4D101EB820022
:10729C0010BD002010BD0000380300202DE9F04186
:1072AC0086B00D4690461F46044603AB4FF6FF7260
:1072BC001B21FEF7F0F8059040B3FF210291024626
:1072CC00BDF80C10DDF834C001910DF11203002152
:1072DC00009120463946E047064688B97889ADF8D2
:1072EC001000E80705D5424604A92046FDF7ADFF7E
:1072FC0005E00C9B424604A92046FDF7B5FF064667
:10730C002EB11B2104A8FEF7D5F800E01526304657
:10731C0006B0BDE8F0810000016809680847036801
:10732C005B681847034A0C2303FB00200268D268F1
:10733C0010470000DCF701000FF218012422FBF7C4
:10734C00D5BF03681B69184701688969084703683A
:10735C00DB69184700000000FFFFFFFFFFFFFFFF86
:10736C0000000000000000000101010100C201004A
:10737C00030000000000000070B504464A48006895
:10738C000D468047064649480FF22902C4604FF467
:10739C000671056101441830FFF760FCFFF7ECFC47
:1073AC003046BDE870404249096808473F480078BC
:1073BC007047000038B50C463C4D0021A980688010
:1073CC00010003D029690A0018BF8847200008D0A3
:1073DC0000202870E968080003D0E88808B9204626
:1073EC008847E988080003D06869BDE8344017E095
:1073FC0031BDF8B504460D4600F047F8A84202D25C
:10740C0000F043F80546294EB788F01900F1180131
:10741C002A462046FBF75AFFE819B0802846F2BDF1
:10742C002DE9F04104462048204E0068204F0D46BF
:10743C0080478046307820B1396840468847002024
:10744C0021E0B5F5007F07DD4FF40070A5F5007164
:10745C0020444FF4007500E00021F18070612A4651
:10746C004FF4067021463018FBF730FF01203070C6
:10747C00B068401CB0602846FFF78FFC05463968A1
:10748C00404688472846BDE8F081084841888088F6
:10749C00081A00F50070011200EBD1514912A0EB53
:1074AC00412080B2704700000C090020882A00207F
:1074BC0010090020F8B52F4C2F4F0546606828188E
:1074CC006060002660884119B1F5007F08DDC0F5C9
:1074DC000076B1B23818FFF78CFF0020AD1B60802E
:1074EC00A9B260883844FFF784FF60882288281886
:1074FC0080B2010A00EBD151490AA0EB4120608017
:10750C007519618840F23910891A8142BCBF6168D3
:10751C00814205DB0120FFF7B9FD1848FEF7CCFBD3
:10752C00A8B2F2BD134841880088081A00F5007013
:10753C00011200EBD1514912A0EB412080B27047EF
:10754C0070B50C4B0C4D1C8800220CE0A4B2521CE4
:10755C002E5D00F8016B641CA4B2260A04EBD6560F
:10756C00760AA4EB462496B28E42EFD31C800846D2
:10757C0070BD0000DC3E002058360020883D002005
:10758C0016B504460A46009401AB69460648784491
:10759C001630FAF755FF009A0021117000285CBFD5
:1075AC000098001B16BD00BF7BA5FFFF2DE9F04F17
:1075BC0085B004461E000D4690461CBF002030606E
:1075CC00A14601E009F1010999F80000A0F10901B7
:1075DC000529F7D32028F5D02D2816BF2B2819F80C
:1075EC00017B2B27B8F1000F57D4B8F1010F54D001
:1075FC00B8F1250F51DAB8F1010F0DDBB8F1100F0E
:10760C0004BF99F80000302802BF99F8010040F03F
:10761C002000782814D10EE099F80000302818BF0B
:10762C004FF00A080CD199F8010040F0200078289E
:10763C0004D14FF0100809F1020901E04FF00808DD
:10764C00CDF8109001E009F1010999F800003028FB
:10765C00F9D00FF2A40B4FF0000ACDF80C908DF876
:10766C0008B00AE09DF80810CDF804A0401AC0B28A
:10767C00009008FB0A0A09F1010999F80010A1F120
:10768C0041001A2838BF203142465846FBF7F2FD1C
:10769C000028E7D10498484503D105B12C6000209F
:1076AC0025E00FF27C01039811F80810A9EB0000FB
:1076BC00401A14D4012808DA0098BAEB000004D35D
:1076CC000199B0FBF8F0884209D000F03DF8222176
:1076DC0001600EB1012030604FF0FF3A03E02D2F16
:1076EC0008BFCAF1000A0DB1C5F80090504605B0AC
:1076FC00BDE8F08F002359E730313233343536375B
:10770C0038396162636465666768696A6B6C6D6E53
:10771C006F707172737475767778797A00000000E7
:10772C0000002115110E0D0C0B0B0A0A0909090991
:10773C0009080808080808080707070707070707C4
:10774C000707070707000000014800F003B8000016
:10775C00C009002070470000DFF800F0ADB5011043
:10776C00DFF800F019AE0110DFF800F085C201104F
:10777C00DFF800F081C20110DFF800F055C10110F4
:10778C00DFF800F043C20110DFF800F079AB011014
:10779C00DFF800F0D9B60110DFF800F0EDB30110FE
:1077AC0020B108232C220021F9F7B2BE704720B17A
:1077BC0008233C220021FCF70FBA704780B5F8F77C
:1077CC000FFFADF80000FAF7A1FAADF8020000982F
:1077DC0002BD01B5BDF80200FAF79CFABDF8000035
:1077EC00BDE80240F8F700BF38B5DFF87448DFF8A1
:1077FC0074580020A4F8FC0FE820208040F6147088
:10780C00A4F8E80004F1E8006860002000F003F838
:10781C00A8606C6031BDF8B500240025061D16F07B
:10782C0003001CBF311D0E1AFFF7C8FFDFF8342808
:10783C00B6B21060112EB4BF576897683A8813041B
:10784C0003D582F4004200251AE02B0014D02388C3
:10785C0039880B4423809BB2B34211D327461A4676
:10786C00B7B1921B92B2042AA7BFBA5346F4004197
:10787C00398841F4004109E0B242F1DA01253C4675
:10788C0017443A88002ADAD1002701E027F8041BB4
:10789C00FFF79FFF3846F2BD10B50446FFF78EFF89
:1078AC00DFF8C017086034F8042CC2F30E0224F879
:1078BC00042C221F4B689A4238BF4A60BDE8104026
:1078CC0087E738B50446FFF779FF00210C23DFF872
:1078DC0098274B43D518AA6C4AB1944204D1FFF7B0
:1078EC0078FF05F1480032BD491C0329EED3FFF7A0
:1078FC0070FF002032BD70B50546FFF75FFF0446F0
:10790C0000200C22DFF8601742438E18B16C49B985
:10791C0000203065B5640022FFF71EFFF06418B933
:10792C0017F068FB8D4205D12046FFF752FF06F198
:10793C00480070BD401C0328E3D32046FFF749FFE5
:10794C00002070BD38B50446FFF738FF0025DFF87E
:10795C0018170C226A438A5A130008D0944203D198
:10796C00FFF737FFA8B232BD6D1C062DF1D3FFF720
:10797C0030FFFF2032BD10B504462088FFF7E2FF30
:10798C00FF2800D16AE10C22DFF8DC1650430844D2
:10799C008168080002D16FF0010010BD2046BDE8DF
:1079AC001040084702460FF2A470104710B5002093
:1079BC000C21DFF8B426002401FB00F31344401C17
:1079CC0003289C641C65F7D30020002301FB00F402
:1079DC00401C13530628F9D3082010800FF2557061
:1079EC009060BDE81040FFE670B590B0F8F7F8FD78
:1079FC0004466846FFF7DBFE0520069000224FF494
:107A0C004870089069464FF201000490DFF85C065C
:107A1C000590DFF85C06FFF7A3FE050006D0FFF724
:107A2C00CDFE06462846FFF766FF08B917F0E2FAC6
:107A3C003046FFF7CEFE2046F8F7D6FD10B070BDED
:107A4C00F8B500F0E5F8FFF756FF0546FFF7B6FE70
:107A5C00A28800210C26DFF810364E4333441E88D2
:107A6C00370007D11A805D60A2689A60A1816968AD
:107A7C002161C4E2B24204D1FFF7ABFE6FF0020009
:107A8C00F2BD491C0629E5D317F0B4FA00BF38B58E
:107A9C0000F0BEF8FFF72FFF050016D0FFF78EFEA3
:107AAC0000210C23DFF8C0254B431A4413884BB933
:107ABC004FF6F8731380556000239360A1806968BA
:107ACC00A16014E7491C0629EBD317F093FA00BF09
:107ADC0010B5044660680C3080B2FFF79CFE10B9FC
:107AEC006FF0030010BD6168018100210160FF216E
:107AFC0081720C30A060002010BD80B540680C383D
:107B0C0010E080B287E610B50446606880B2FFF7DB
:107B1C0082FEA06000280CBF6FF00300002010BD97
:107B2C0080B54068FFF7B8FE002002BD38B50446AA
:107B3C000D46FFF743FE002145F80C1C216811B9D6
:107B4C00256006E0114651F80C2C002AFAD141F8B8
:107B5C000C5CBDE832403CE62DE9F04104466FF088
:107B6C000206E068A0F10C05E0880628BCBFA088DE
:107B7C0006280BDAFFF722FEE188DFF8EC840C27ED
:107B8C0079434144496819B9FFF723FE304617E0A1
:107B9C00FFF71FFEA0882871E0886871207AA87111
:107BAC00E088E1687843404440680830FFF7BEFF46
:107BBC00E0887843404440684068FCF711F80020A6
:107BCC00BDE8F08170B500F023F8FFF77AFE0600EF
:107BDC0002D16FF0040070BDFFF7F0FDB168002515
:107BEC0041B10D46A5F10C010A68B26000220A6091
:107BFC00FF228A72FFF7EDFDA560A5F10C010DB90E
:107C0C00022070BD0879A0804879E080002070BD0A
:107C1C000446F8F7EDBC06280ADA0C23DFF84824F2
:107C2C005843105A02001CBF4FF6F872904202D112
:107C3C004FF0FF307047088000207047811D80880E
:107C4C00E9E710B50446E088FFF77CFEFF2800D179
:107C5C0004E0E0802046BDE810407DE74FF0FF30A7
:107C6C0010BD3EB50446FFF7ADFF050017D1A08847
:107C7C006946FFF7D0FF78B1A06802900821ADF8F3
:107C8C00041001A80321ADF80610DFF8E813896889
:107C9C0088476FF005003EBDBDF80000A080284667
:107CAC003EBD10B5DFF8D02312680C464FF47A7144
:107CBC00A1FB00010023FAF7B7FA002399424FF019
:107CCC00004201D8904202D36FF0020010BD206038
:107CDC00002010BD38B5FFF79BFFFFF7F2FD0546FE
:107CEC00F8F7DEFC002818BF012800D015B96FF09A
:107CFC00040032BD606840B9009000996868FDF7D7
:107D0C0063FD401E8041C00F32BD10F1010F08BF52
:107D1C004FF0FF30F0D000F04EF90028EDD032BD1E
:107D2C0080B54068FBF75CFF002002BD17F062F9DC
:107D3C0000BF80B54068FFF717FD002002BD80B57D
:107D4C004068FFF715FD002002BD80B5FFF714FD5C
:107D5C00FFF716FD002002BD80B5F8F741FCF9F7DE
:107D6C00D5FF002002BD10B58CB004466846FFF765
:107D7C0017FDE02000F013F808B917F03BF90BE001
:107D8C0010B58CB004466846FFF70AFDE06800F0B9
:107D9C0006F808B917F02EF900200CB010BD0890A9
:107DAC000023A16860686A46FFF7EEBC10B5044674
:107DBC00FFF7EEFC6060002010BD01468868496842
:107DCC000847F0B507468BB0BC68AA4D6CBB0C20BD
:107DDC00FFF721FD04006FF003061ED008232422B8
:107DEC00002101A8FDF72AFF0020ADF81400069031
:107DFC00079400237968A14801AAFFF7CDFC206005
:107E0C0068B90820ADF800000C20ADF802006846F7
:107E1C00A96888472046FFF73FFD304618E0F86810
:107E2C0060603869A060BC600AE02868804706463C
:107E3C002068F8F7E1FB3869A0603046696888472C
:107E4C0079682068F8F7DCFB2068F8F7DDFB002088
:107E5C000BB0F0BD10B5044682B0606800F0ABF812
:107E6C0020B9009860602046FFF7ABFF16BD80B5C7
:107E7C00406810B96FF0020002BD0068F8F7BCFB57
:107E8C00002002BD7C49096841600020704750B554
:107E9C000446794802686FF00046A6FB02010023F5
:107EAC004FF47A72FAF7C0F9002399424FF000426E
:107EBC0001D8904200D330466060002050BD2DE9BF
:107ECC00F04186B00646F8F793FBFFF7FAFC044640
:107EDC00002002900025F8F7E3FB002818BF0128CA
:107EEC0000D014B96FF0040062E0706820B110F19A
:107EFC00010F03D14FF0FF30009003E000F05BF86E
:107F0C00070054D1FFF744FC0099012701EB00084E
:107F1C0000E0009000996068FDF756FC78B303A868
:107F2C00FFF750FE07001AD1BDF8100001A9FFF7AA
:107F3C0072FE80B9059ABDF81210BDF80400B36842
:107F4C00984740B1BDF80400B081BDF81200F08133
:107F5C000598306113E0059902A8FFF7E7FD00983A
:107F6C0001276D1C10F1010F18BF0028D2D0FFF7AC
:107F7C000FFCB8EB000002D000998142C9D2029EDE
:107F8C00FFF71CFC56B1314600E0114651F80C2CA1
:107F9C00002AFAD1A26841F80C2CA660FFF719FC54
:107FAC00002D03E06068FBF71BFE6D1EFAD138460E
:107FBC0006B0BDE8F081694673E6F8B5FFF728FE18
:107FCC000546F8F76DFB002818BF01286FF0040672
:107FDC0013D0FFF7F3FB0021234A0C234B43D75A52
:107FEC004FB113445B681B68AB4201D1A18006E022
:107FFC00491C0629F1D3FFF7ECFB3046F2BDFFF725
:10800C00E8FB0020F2BDF8B50446F8F749FB002860
:10801C0018BF012802D16FF00400F2BDF8F7E8FA9E
:10802C000546FFF7CBFB00210F4A0C234B43D65AD6
:10803C0037000ED0A788BE4208D1D118496809680C
:10804C00A9420CBF01210021A160D8E7491C0629D7
:10805C00EBD3FFF7BEFB4FF0FF30F2BD000000008A
:10806C00D4090020A03E00209823002034080020D2
:10807C00B17900000C090020208E0000C77D0000A3
:10808C0070B504463C20FFF7C6FB05006FF00306F5
:10809C0011D0FFF78CFB207AA8610022608928623E
:1080AC002946E06828616068FFF75AFB04462846B9
:1080BC00FFF7F2FB0CB9304670BD002070BD70B5F7
:1080CC0004462420FFF7A7FB05006FF0030613D02E
:1080DC00082324220021FDF77BFB2079012808BF0F
:1080EC002876A06800222946FFF736FBE060284678
:1080FC00FFF7D2FBE06808B9304670BD002070BDB8
:10810C0010B5044682B0A06840B900900099606830
:10811C00FDF75AFB401E8041C00F16BD10F1010F38
:10812C0008BF4FF0FF30F0D0FFF745FF0028EDD02F
:10813C0016BD00004188292902D36FF00100704759
:10814C000FF2140252F82110084700008379000046
:10815C00C9770000DF7700004D7A00009B7A0000A1
:10816C00DD7A0000077B0000137B00002D7B0000F4
:10817C00657B0000D17B00004F7C00006F7C000011
:10818C00E17C00002D7D0000397D00003F7D00006A
:10819C004B7D0000577D0000657D0000737D000065
:1081AC00B97D0000617E0000917E00009B7E000086
:1081BC00497C0000D1F401009BF50100CB7E00004E
:1081CC00C77F0000CF7D00007B7E000035F50100ED
:1081DC006DF5010081F5010013800000D1F501005F
:1081EC00EDF501008D800000CB8000000D810000BA
:1081FC00E3F50100FBF501008D7D0000DFF800F0D8
:10820C0061C20110DFF800F0E1C20110DFF800F0EC
:10821C00B9C20110DFF800F0F9BF01108069C00885
:10822C0000F00100704750F8382F1143016070477F
:10823C0050F8382F22EA0101016070474164704701
:10824C00406800F00F007047002141607047817B4F
:10825C00FF291CBFC07BFF2801D0012070470020E4
:10826C00704738B5F9F752FDDFF8B4570446287853
:10827C0020B90420F8F7EAFC012028700CE038B58E
:10828C00F9F744FDDFF898570446287820B104200C
:10829C00F8F7FAFB002028702046BDE83240F9F7C9
:1082AC0039BD40687430FBF79BBC40689030FBF7DD
:1082BC0097BC70B5446885680E4606E0206A401C81
:1082CC002062761E606A401C60624EB1206ADFF844
:1082DC005427126801782868926990470028EDD1DC
:1082EC00304670BD70B5456886680C4608E0296B51
:1082FC000870641E286B401C2863686B401C686304
:10830C0044B1DFF82017096830680969884710F113
:10831C00010FECD1204670BD70B504466568A668A7
:10832C00FFF7ADFF00F0E2FAD7E270B5446804F154
:10833C00AC050E462846F8F75FF90FF24871627FDC
:10834C00207F51F822100818C01D7043DFF8D81692
:10835C004843A169B0FBF1F0DFF8D016096864302E
:10836C00B0FBF1F12846F8F74BF92846BDE8704010
:10837C00F8F74AB9F8B504466568A66805F1AC0784
:10838C003846F8F739F93068FFF748FF88B1DFF85D
:10839C009C1609684FF4FA70B0FBF1F1022938BF52
:1083AC0001213846F8F72CF93846BDE8F240F8F7C9
:1083BC002BB9FFF764FF30682021FFF739FF00F07D
:1083CC0031FA25E270B504460D4620212868DFF805
:1083DC006066FFF72DFF297B30680122FDF7B1FBAA
:1083EC00297B30680122FDF7C9FB297B306800220C
:1083FC00FDF7EBFBA97B30680022FDF7E6FBA078CC
:10840C00012805D12868FFF709FF0028FAD105E0FB
:10841C004FF0FF3104F17400FDF7D6F9297B306879
:10842C001022FDF7D2FB2846FFF711FF30B1A97BD4
:10843C003068BDE870401122FDF7C7BB70BD2DE957
:10844C00F8438146D9F808603068D9F80470046C98
:10845C002146FFF7F3FE14F4F06F07F128052DD039
:10846C00600510D53068FFF7EBFE80463068FFF7EB
:10847C00EBFE2969212928BF202100F050F817E0D4
:10848C002869401E2861286990B1012100F047F845
:10849C003068FFF7D5FE80463068FFF7D5FEB8F19F
:1084AC00000FEDD0A868401EA860E868401EE86088
:1084BC0087F81F80484600F0F9F91FE060060BD5DD
:1084CC00296900F02CF82861687910B10020286126
:1084DC0011E0286900280DE0E0060FD5287D471E25
:1084EC002869874228BF0746394600F018F82869E2
:1084FC00C01B286102D14846FFF70EFFA0060CD521
:10850C002C6854B121464846FFF7D3FE286020B9A9
:10851C00211D4846BDE8F44307E7BDE8F183484612
:10852C00E0E64068002101700020DFF8F4140870C8
:10853C007047F0B504466568A76897B00E46F9F722
:10854C00E5FB297800294CD101212970F9F7E2FBD0
:10855C001EB90DA8FEF7F0FE0DAE3078687070787D
:10856C00A87070686860B068A860F068E8603069EE
:10857C002861307D2875707D6875B07DA875B069EF
:10858C00A861307F2877707F6877B07FA87700204C
:10859C002862286368626863A862A86385F82C0067
:1085AC0085F82D00102085F83C00002085F83D0052
:1085BC00B868C0B2F8F7F4FA204600F0A0F92046EB
:1085CC0000F0F2F988B9DFF85C1409683868C968FA
:1085DC008847B868C0B2F8F777FAF9F797FB00212B
:1085EC002970F9F797FB00204DE008233022002179
:1085FC0001A8FDF7F1F800200694009001AB796812
:10860C00DFF8302405F15800FDF7EAF8082324229E
:10861C00002101A8FDF7DCF801208DF81C00A878DA
:10862C0040B901AA002105F17400FDF7DDF8DFF86F
:10863C0008042861687840B901AA002105F190006E
:10864C00FDF7D2F8DFF8F403E860082324220021B8
:10865C0001A8FDF7F3FA00200690ADF8140007947A
:10866C0001AB0A22DFF8D81305F1AC00FDF7EEFAE6
:10867C000020009023460FF2D932042105F144006A
:10868C00F8F779FA204617B0F0BD38B5446885681C
:10869C00DFF89C030068FDF740FA286840F2F2719D
:1086AC00FFF7C6FDDFF87C1309682868C96888479E
:1086BC00A868C0B2F8F708FA04F15800FFF79EFD5D
:1086CC00A07818B904F17400FFF79CFD607818B914
:1086DC0004F19000FFF796FD04F1AC00FFF796FD56
:1086EC00F9F714FB00212170F9F714FB04F1440095
:1086FC00BDE83240F8F7C8BB426820296FF0010092
:10870C0002D0212905D07047012082F82D000020CD
:10871C007047002082F82D0070472DE9F84304467D
:10872C006668A7680D469146F9F7F0FA8046B06A7C
:10873C0018B14046F9F7EEFA38E006F1AC00F7F75D
:10874C005BFF0020F077356270624046F9F7E2FA81
:10875C00FFF787FDBB48016841F48071016020463A
:10876C004946FFF7A6FDB06248B949462046FFF7D7
:10877C00DCFDB078F8B900F021F8D0B90DE038681C
:10878C002021FFF750FDB078A8B900F017F880B998
:10879C0049462046FFF7C9FD0020B062394610203B
:1087AC00F0773046FFF70EFEFFF769FD4FF0FF3014
:1087BC0002E0706A00E00020BDE8F283B16806F1C7
:1087CC007400FDF701B86EE0F8B500F093F80746B9
:1087DC00A86A40B93068FFF721FD20B93846BDE8DA
:1087EC00F240F9F797BA0020A8623846F9F792FAE6
:1087FC003046FFF72CFD18B131462846FFF7E2FD55
:10880C0030682021FFF714FD00F00CF8FFF737FD5E
:10881C006A6A286A2B69811A2962204601B0BDE870
:10882C00F04018478748016821F480710160704757
:10883C00F8B5446885680E461746F9F767FAA16BD8
:10884C0021B1F9F767FA4FF0FF30F2BDE1776163C0
:10885C00A7632663F9F75EFAFFF703FD7948016811
:10886C0041F4007101604FF4FA612868FFF7DBFCFA
:10887C006078A8B9616804F19000FCF7A5FF68B9AD
:10888C00A0634FF4FA612868FFF7D2FCFFF7F7FCFE
:10889C00206B616B401A20631020E077606BF2BD97
:1088AC000020F2BD00BF4FF0FF30704770B500F0F4
:1088BC0021F8A96B002904BFBDE87040F9F72ABA6A
:1088CC000021A963F9F726FA00F010F85D48016859
:1088DC0021F400710160FFF7D2FC6A6B286BEB6826
:1088EC00811A29632046BDE87040184730684FF460
:1088FC00FA619DE404466568A668F9F707BAF0B515
:10890C0087B0044602A80FF25811464E1422FAF70B
:10891C00EDFC6568A46831682068C968884740F236
:10892C00F27720683946FFF783FC20683946FFF759
:10893C0085FC05F13C0002AA41780078C00852F889
:10894C00200008432168486300A8FFF763FC05F189
:10895C0018000FF22011027951F822100FF2241294
:10896C00437952F82320837935686D6811430FF2EF
:10897C001C1252F8232042EA010302680199206874
:10898C00A847314D286840F010002860686840F016
:10899C00010068602046FFF75AFC18B1686840F483
:1089AC004040686007B0F0BDF0B58468274D607B2F
:1089BC0085B040F00040009000AE207B28437060F2
:1089CC0008272046FFF743FC38B1A07B40F000405D
:1089DC00B0601027E07B2843F060FF20B85100A95D
:1089EC00134D281DFDF734F82860B8B1617B0F22B8
:1089FC00FDF7EBF8217B28681022FDF7E6F82046FE
:108A0C00FFF725FC48B1A17B28681122FDF7DDF8A2
:108A1C00E17B28681222FDF7D8F8012005B0F0BDE3
:108A2C00363F0020D001001040420F00208E000085
:108A3C00903E00204B840000AF820000B782000003
:108A4C0081830000301000402C1000400000C0A0BA
:108A5C0080B5042804BF0846FFF751FF002002BD73
:108A6C0000000000080000001000000018000000CA
:108A7C00200000000000000020000000400000006A
:108A8C006000000000000000080000000000000072
:108A9C0006000000020000008600000082000000BA
:108AAC00F56B010064350000D409002000000000C3
:108ABC001F6801000200000002000000A803000073
:108ACC001B000000780100202C000000036801004E
:108ADC0002000000020000007375FFFF030000009D
:108AEC00EC01002004000000E76701000200000018
:108AFC00020000005175FFFF03000000F001002090
:108B0C0008000000CB67010002000000020000001A
:108B1C006F0300001A000000A401002024000000D4
:108B2C00AF67010002000000020000000475FFFFA7
:108B3C000C000000C80100201C000000936701001D
:108B4C000200000002000000DC0200001C0000001B
:108B5C0000010020440000007767010002000000C3
:108B6C0002000000EA74FFFF060000000002002073
:108B7C00040000005B67010002000000020000001E
:108B8C00C874FFFF03000000F8010020080000007B
:108B9C003F6701000200000002000000A402000078
:108BAC002400000044010020340000002367010071
:108BBC0002000000020000008474FFFF09000000A6
:108BCC00E40100200800000007670100020000001B
:108BDC0002000000C5020000700300000802002023
:108BEC00CA0700000A18232A242A252A262A272AFB
:108BFC00282A292A2A2A502A02000000F08B000079
:108C0C0000F00BF8002803D016F016FE16F042FE0A
:108C1C00002016F063FDF9F79DF801207047000065
:108C2C001800000000000000000000003C8C000058
:108C3C0008000000000000007661722530326420CC
:108C4C00252D32352E3235733D2025730D0A00004B
:108C5C0000B581B016F018FEC046C04601B05DF8F4
:108C6C0004EBFFF7CDBF000044F2E830C2F2000085
:108C7C00854648F65D40C0F200008047FEE70000E4
:108C8C0001000000000000000000000000000000D7
:108C9C0001000000446973636F7665727950656EEC
:108CAC0064696E67000000002D424C452D436F6EC9
:108CBC006E656374696F6E55700000002D424C45F3
:108CCC002D436F6E6E656374696F6E446F776E00C3
:108CDC002D424C452D4279706173734D6F64652D37
:108CEC000000000045B50110BD1E000099A6011042
:108CFC0019B801106C65646973636F6E6E6563748B
:108D0C00000000002D436F6D6D616E644D6F6465E6
:108D1C002D000000526573657450656E64696E6752
:108D2C0000000000436F6E6E65637454696D656F6F
:108D3C00757400004244416464726573733A257320
:108D4C000D0A000000280000032800000129000083
:108D5C0002290000666163746F7279696E69740030
:108D6C006C6562797061737300000000436F6E660E
:108D7C0069674F6B00000000436F6E666967457250
:108D8C00726F72002D536C6565704D6F64652D00AC
:108D9C0041542D41422025730D0A000061742B6152
:108DAC0062200000636F6E66696700007265736510
:108DBC0074000000736C6565700000004164764FB0
:108DCC006B0000000A0B0C0D0E0F00005E235E24DE
:108DDC005E2500002D412D0D0A0000002D422D0DA9
:108DEC000A0000002D432D0D0A0000002D442D0D0E
:108DFC000A000000100000005000000008000000F5
:108E0C008F0900004B00000064000000820000008D
:108E1C00200000000A00000004000000190F0000F0
:108E2C000D0A000083010001A10CD003D80700201B
:108E3C00000143BC091420023401002004523C04FC
:108E4C001200011003303F002024041228042110CA
:108E5C0022E8082304000190082001010000283BAF
:108E6C00002000015200011007C8060020780700FE
:108E7C00200111C30100011003C8050020082022A5
:108E8C00000150026CDC02000150032C070020038F
:108E9C000D1003531E00008D04100702000000503B
:108EAC008D000001082002048C0000105254102088
:108EBC0002C60900201043F28B10435C04106120A1
:108ECC0052C72052F420D2642052C82052F620D22D
:108EDC007C2052C92052F820D2942052CA2052FA37
:108EEC0020D2AC2052CB2052FC20D2C42052CC2019
:108EFC0052FE20D2DC2052CD2043008C10D2F42024
:108F0C0052CE2052022010020405002007B00201AC
:108F1C0000030001F00B9A3075FFFF0600800C0077
:108F2C0000E8030001F0013C020106AF560E44615B
:108F3C0055A00A4D6F64656C204E756D6265726943
:108F4C00F00302536572696119500F4669726D77AF
:108F5C00617265205265766973696F6E1CF002034D
:108F6C004861726418F00203536F667418500F4D09
:108F7C00616E756661637475726572204E616D65A4
:108F8C00181003FE006578707C14046D656E7461B6
:108F9C006CC9120D19F4020A100100140629006D97
:108FAC002003BC0114F80120031ACF201210085220
:108FBC0004184B140530125C202909521010525819
:108FCC0030CB880860C3D00920D2A020D2D1204752
:108FDC00B8085C210C12C05C210412E804879C01C7
:108FEC00746101438D0912F0040108060020C805C4
:108FFC002043DD1E12213C2144131027B0422714BC
:10900C0021605291401207E1100B384035002D4081
:10901C000140028460005D08102700F80118A38449
:10902C00070083057EA40306E0EA2306010088609E
:10903C004500C300380103040102638400007384FB
:10904C003800352C100F08047F17AC526003A302B4
:10905C00AD0163026801FF01127C94837C06CC2174
:10906C00016204A111F14358381CE0020BC201103B
:10907C00B8F301010001A11443C5A70D52A5E021CD
:10908C001EC00460070020C5A73961106108834029
:10909C00022041501001010024382104F1031C224C
:1090AC00401886075847B110F4B001FF002C6963D3
:1090BC00411418496612783421049EE57B0312058D
:1090CC000BE5A152D05C12A808210452B00452B88E
:1090DC000452C00452C80452D00452D80452E004C2
:1090EC0052E80452F00452F804430008041A105CCD
:1090FC001220041EA0E40412780812840412B40C8A
:10910C0012C80412DC041290101230042AC8841401
:10911C00020F1B0928B81FC4F7030511D513FC3E19
:10912C0044F402023F00202C955407FF400080FFBE
:10913C00088080FF30F107011C07446174612043F3
:10914C00686172B0031D9B03300273746963F8F09D
:10915C0004015374617475731AF00401436F6E66E5
:10916C00696718100A53696D706C6520424C452074
:10917C0050162C0270686572E3031300CC7B120846
:10918C000847082450438006103005072000C00211
:10919C0000C0A01003C9770000DF041783798C206E
:1091AC00051210001000020A2C31C051C41AC9500B
:1091BC0040042D1F00008F1FCB25BF1D40051C0434
:1091CC000302E0C0004CA8032104525404525C0476
:1091DC00526404526C04527404527C04528404523F
:1091EC008C04529404529C0452A40416A87C6C0A5D
:1091FC002C8E0000394400002F4500003C03600118
:09920C00FFFF0201000114020A37
:020000040001F9
:10F00000012000F001B8000020210903263118205A
:10F01000ABBEF9E74275696C6456657273696F6ED1
:10F0200000000000424C455F323031363038303815
:10F030004200000042445F414444520030303034CA
:10F040003365323630306132000000004465766945
:10F0500063654E616D650000426C655F5065726965
:10F0600070686572616C000055617274426175640C
:10F0700072617465000000003131353230300000BB
:10F0800055617274446174614269747300000000D8
:10F09000380000005561727453746F704269747364
:10F0A0000000000031000000486F73744465657013
:10F0B000536C656570456E0030000000486F7374D6
:10F0C0004576656E74730000426441646472456EF7
:10F0D00062000000416476496E744D696E00000064
:10F0E00033320000416476496E744D61780000004F
:10F0F0005363616E496E74005363616E57696E6449
:10F100006F77000031380000436F6E6E656374499D
:10F110006E744D696E00000031360000436F6E6EF4
:10F12000656374496E744D617800000053657276B2
:10F1300069636555554944004630303043304531A8
:10F140002D303435312D343030302D423030302DAB
:10F15000303030303030303030303030000000006F
:10F160000000000014F0010024F001000400000081
:10F170000100000034F001003CF001000400000038
:10F18000020000004CF0010058F0010004000000F3
:10F190000300000068F0010078F0010000000000AA
:10F1A0000400000080F0010090F001000000000069
:10F1B0000500000094F00100A4F001000000000030
:10F1C00006000000A8F00100B8F0010000000000F7
:10F1D00007000000BCF00100A4F0010000000000E6
:10F1E00008000000C8F00100B8F0010000000000B5
:10F1F00009000000D4F00100E0F001000000000070
:10F200000A000000E4F00100E0F00100000000004E
:10F210000B000000F0F00100E0F001000000000031
:10F220000C000000F8F0010004F1010000000000F3
:10F230000D00000008F1010018F1010000000000BD
:10F240000E0000001CF1010018F101000000000098
:10F250000F0000002CF1010038F101000000000057
:10F2600001680A680A4482604B681A44C260083127
:10F27000016070478168C268914208D101680A68DC
:10F280000A4482604B681A44C26008310160816898
:10F29000491C816011F8010D704738B504460D46D0
:10F2A000A068E168884212D120686168884208BF7E
:10F2B000FFF7A6FE2068227C016802B14944A160E4
:10F2C00042680A44E260083091422060ECD0A068B5
:10F2D000401CA06000F8015D31BD2DE9F0418AB00D
:10F2E00000F1080105910268520801EBC201069184
:10F2F0000021079108910168490800EBC10108311C
:10F300000091017901F001018DF810104068009919
:10F31000400801EBC000019000200290039006E03D
:10F3200005A8FFF79DFF07980899884207D105981F
:10F3300006998842F4D101980AB0BDE8F08105A889
:10F34000FFF798FF044614F0030603D105A8FFF762
:10F3500091FFC61C25090F2D14D105A8FFF78AFFC0
:10F3600000F10F050EE007980899884204BF05A830
:10F37000FFF776FF0798401C079010F8011D6846BC
:10F38000FFF78BFF761EEED1002DCCD005A8FFF73E
:10F3900071FF0646A00800F00300032804BF05A87B
:10F3A000FFF768FFDDF800800299039F06EB00205D
:10F3B00008E0A8F10808A8F10801801A0A6849685D
:10F3C0005718394658F8082C8A1A8242F1D340421D
:10F3D0000C18AE1CA7D0BC4206D158F8044B58F804
:10F3E000040B2718BC42F8D00298039914F8015B6B
:10F3F000884217D100980199884208BFFFF700FEA4
:10F40000009800689DF81010029009B148440290DD
:10F41000009902984968009A014408328842039191
:10F420000092E7D00298401C0290761E00F8015D21
:10F430003FF479AFCFE7000080B501280BD0022858
:10F440000BD0042802D0082809D00AE000200A685E
:10F450009047002002BD0220F9E70420F7E70520CD
:10F46000F5E7FFF7CDFD00BF38B50446012504E000
:10F4700005FA00F0C0B2E1F7EFFBB4FA84F02028FF
:10F4800000D131BD00F01CF8F2DB401FC0B2E1F743
:10F490008DFBF2E738B50446012504E005FA00F0DB
:10F4A000C0B2E1F7F7FAB4FA84F0202800D131BDF8
:10F4B00000F006F8F2DB401FC0B2E1F70BFBF2E709
:10F4C000C0F11F00C0B205FA00F14C40052870479A
:10F4D00038B500793C4CA8B1E8F776F905462078B4
:10F4E000FF2805D12846E8F77AF96FF0060032BD0B
:10F4F000401C2070C0B2012804BF6068FFF7B4FF51
:10F50000284613E0E8F760F921780A0004D1E8F70B
:10F5100066F96FF0070032BD491E2170C9B229B9E2
:10F52000E8F75DF96068FFF7B5FF01E0E8F757F924
:10F53000002032BD70B50446606810F07F4F02D0E5
:10F540006FF0020070BDE8F73FF91F4E05463078B6
:10F5500028B17068FFF79EFF6068FFF785FF60685D
:10F5600070602846E8F73BF9002070BD80B5406820
:10F5700010F07F4F00D00DE0FFF776FF002002BDB6
:10F5800080B5406810F07F4F00D003E0FFF782FFA6
:10F59000002002BD6FF0020002BD1CB50446A16848
:10F5A000606808601420E8F7B2FA019010B96FF0B3
:10F5B000030016BD002000900F21A3680198034AA4
:10F5C000E1F7DFFA002016BD3C09002039F4010004
:10F5D00010B50446E1F74AFA00B10120207100207D
:10F5E00010BD80B5E1F742FC002002BD10B5044615
:10F5F000E1F735FA6060002010BD10B50446606880
:10F60000E1F732FAA060002010BD00007B756E6B40
:10F610006E6F776E2D696E7374616E63652D6E61AA
:10F620006D657D007B656D7074792D696E73746195
:10F630006E63652D6E616D657D0000007B73746186
:10F640007469632D696E7374616E63652D6E616D8F
:10F65000657D00008F3F00008F3F01008F3F02005B
:10F660008F3F0300903F00018F3F0101903F000258
:10F67000903F00038F3F01048F3F00058F12080465
:10F680008F3F00048F3F0006513F00007F3F010085
:10F690003F3F04003F3F02003F3F01007F3F020029
:10F6A00019E050F8041BCB0744BFA9F10103591816
:10F6B000121F0023042A41F8043BF9D25FEA827C3E
:10F6C0000B4604D54FF0000CA1F800C09B1CD107DD
:10F6D00044BF0021197050F8042B002AE1D1704773
:10F6E000DFF800F055C0011080B50B48E6F70CF9C3
:10F6F0000420E1F7B1FA0820E1F7AEFAE8F75CF987
:10F70000E8F778F9E6F76EFDE7F70EFCE4F718FB8B
:10F71000FFF7E6FF002002BD000900205379737453
:10F72000656D20436F6E66696775726174696F6E8F
:10F730002053657474696E6773202D20566572734B
:10F74000696F6E20312E300D0A000000B08D000070
:10F7500079490000B88D0000774B0000608D0000F3
:10F760002B4A0000008D00006F4B0000C08D000090
:10F77000874B00006C8D0000974B00007FC8011084
:10F78000C9BC011051B2011037C20110BDAD01104A
:10F79000C1B10110E909000071BA011069BB011083
:10F7A00021C00110EBC70CEEC910F1CB14F4CE143C
:10F7B000F74F21FA5429FD5C35006C56011F6A028F
:10F7C000299C0000A4F701000A0700000010004077
:10F7D00015000000060000000201FFFF1CF80100F8
:10F7E000583A0020CCF701000000000000000000A3
:10F7F0000000000000000000000000B000405104C4
:10F80000E0C000F000000000000000B00040510423
:10F81000E1C000F010000000F4F70100978600003E
:10F82000058700002F8500003F8500003D8800000F
:10F83000B1880000B988000027870000D387000046
:10F84000D587000010B5074979441831064C7C442F
:10F85000163404E00A68081D114488470146A14295
:10F86000F8D110BD4892FEFF8893FEFFFFFFFFFF17
:10F870007C090020040000000000000000000000DF
:10F88000140000002C8C000018000000DFF800F0CD
:10F8900059C501100548012808BFE2F7C2BA7047F0
:10F8A0000348012808BFFFF7F1BF704701000000BF
:04F8B0000100000053
:10FFA80000008006100082FFFDFF58003AFFBFF3F3
:10FFB800FFFFFFFFFFFFFFFFFFFFFFFFFFFFFFFF49
:10FFC800FFFFFFFFFFFFFFFFFFFFFFFFFFFFFFFF39
:10FFD800C505FEC5FFFFFFFFC5FFFFFFC5C5C5FF80
:10FFE800C5C5C5FF00000000FFFFFFFFFFFFFFFFC3
:08FFF800FFFFFFFFFFFFFFFF09
:0400000500008C75F6
:00000001FF
